Component: ARM Compiler 5.06 update 5 (build 528) Tool: armlink [4d35e2]

==============================================================================

Section Cross References

    startup_mk64f12.o(RESET) refers to startup_mk64f12.o(.text) for Reset_Handler
    startup_mk64f12.o(RESET) refers to lwip_dhcp_bm.o(i.SysTick_Handler) for SysTick_Handler
    startup_mk64f12.o(RESET) refers to fsl_enet.o(i.ENET_1588_Timer_IRQHandler) for ENET_1588_Timer_IRQHandler
    startup_mk64f12.o(RESET) refers to fsl_enet.o(i.ENET_Transmit_IRQHandler) for ENET_Transmit_IRQHandler
    startup_mk64f12.o(RESET) refers to fsl_enet.o(i.ENET_Receive_IRQHandler) for ENET_Receive_IRQHandler
    startup_mk64f12.o(RESET) refers to fsl_enet.o(i.ENET_Error_IRQHandler) for ENET_Error_IRQHandler
    startup_mk64f12.o(.text) refers to startup_mk64f12.o(FlashConfig) for FlashConfig
    startup_mk64f12.o(.text) refers to startup_mk64f12.o(RESET) for __Vectors
    startup_mk64f12.o(.text) refers to system_mk64f12.o(i.SystemInit) for SystemInit
    startup_mk64f12.o(.text) refers to entry.o(.ARM.Collect$$$$00000000) for __main
    startup_mk64f12.o(.text) refers to fsl_uart.o(i.UART0_RX_TX_DriverIRQHandler) for UART0_RX_TX_DriverIRQHandler
    startup_mk64f12.o(.text) refers to fsl_uart.o(i.UART1_RX_TX_DriverIRQHandler) for UART1_RX_TX_DriverIRQHandler
    startup_mk64f12.o(.text) refers to fsl_uart.o(i.UART2_RX_TX_DriverIRQHandler) for UART2_RX_TX_DriverIRQHandler
    startup_mk64f12.o(.text) refers to fsl_uart.o(i.UART3_RX_TX_DriverIRQHandler) for UART3_RX_TX_DriverIRQHandler
    startup_mk64f12.o(.text) refers to fsl_uart.o(i.UART4_RX_TX_DriverIRQHandler) for UART4_RX_TX_DriverIRQHandler
    startup_mk64f12.o(.text) refers to fsl_uart.o(i.UART5_RX_TX_DriverIRQHandler) for UART5_RX_TX_DriverIRQHandler
    system_mk64f12.o(i.SystemCoreClockUpdate) refers to system_mk64f12.o(.data) for SystemCoreClock
    fsl_phy.o(i.PHY_EnableLoopback) refers to fsl_phy.o(i.PHY_Read) for PHY_Read
==============================================================================

Removing Unused input sections from the image.

    Removing system_mk64f12.o(.rev16_text), (4 bytes).
    Removing system_mk64f12.o(.revsh_text), (4 bytes).
    Removing system_mk64f12.o(.rrx_text), (6 bytes).
    Removing system_mk64f12.o(i.SystemCoreClockUpdate), (452 bytes).
    Removing fsl_phy.o(.rev16_text), (4 bytes).
    Removing fsl_phy.o(.revsh_text), (4 bytes).
    Removing fsl_phy.o(.rrx_text), (6 bytes).
    Removing fsl_phy.o(i.PHY_EnableLoopback), (166 bytes).
    Removing pin_mux.o(.rev16_text), (4 bytes).
    Removing pin_mux.o(.revsh_text), (4 bytes).
    Removing pin_mux.o(.rrx_text), (6 bytes).
    Removing board.o(.rev16_text), (4 bytes).
    Removing board.o(.revsh_text), (4 bytes).
    Removing board.o(.rrx_text), (6 bytes).
    Removing clock_config.o(.rev16_text), (4 bytes).
    Removing clock_config.o(.revsh_text), (4 bytes).
    Removing clock_config.o(.rrx_text), (6 bytes).
    Removing clock_config.o(i.BOARD_BootClockVLPR), (92 bytes).
==============================================================================

Image Symbol Table

    Local Symbols

    Symbol Name                              Value     Ov Type        Size  Object(Section)

    RESET                                    0x00000000   Section     1024  startup_mk64f12.o(RESET)
    ../../../../../../../devices/MK64F12/arm/startup_MK64F12.s 0x00000000   Number         0  startup_mk64f12.o ABSOLUTE
    ../../../../../../../devices/MK64F12/drivers/fsl_clock.c 0x00000000   Number         0  fsl_clock.o ABSOLUTE
    ../../../../../../../devices/MK64F12/drivers/fsl_common.c 0x00000000   Number         0  fsl_common.o ABSOLUTE
    ../../../../../../../devices/MK64F12/drivers/fsl_enet.c 0x00000000   Number         0  fsl_enet.o ABSOLUTE
    ../../../../../../../devices/MK64F12/drivers/fsl_flash.c 0x00000000   Number         0  fsl_flash.o ABSOLUTE
    ../../../../../../../devices/MK64F12/drivers/fsl_gpio.c 0x00000000   Number         0  fsl_gpio.o ABSOLUTE
    ../../../../../../../devices/MK64F12/drivers/fsl_smc.c 0x00000000   Number         0  fsl_smc.o ABSOLUTE
    ../../../../../../../devices/MK64F12/drivers/fsl_uart.c 0x00000000   Number         0  fsl_uart.o ABSOLUTE
    ../../../../../../../devices/MK64F12/system_MK64F12.c 0x00000000   Number         0  system_mk64f12.o ABSOLUTE
    ../../../../../../../devices/MK64F12/utilities/fsl_debug_console.c 0x00000000   Number         0  fsl_debug_console.o ABSOLUTE
    ../../../../../../../middleware/lwip_2.0.0/port/ethernetif.c 0x00000000   Number         0  ethernetif.o ABSOLUTE
    ../../../../../../../middleware/lwip_2.0.0/port/sys_arch.c 0x00000000   Number         0  sys_arch.o ABSOLUTE
    ../../../../../../../middleware/lwip_2.0.0/src/api/api_lib.c 0x00000000   Number         0  api_lib.o ABSOLUTE
    ../../../../../../../middleware/lwip_2.0.0/src/api/api_msg.c 0x00000000   Number         0  api_msg.o ABSOLUTE
    ../../../../../../../middleware/lwip_2.0.0/src/api/err.c 0x00000000   Number         0  err.o ABSOLUTE
    ../../../../../../../middleware/lwip_2.0.0/src/api/netbuf.c 0x00000000   Number         0  netbuf.o ABSOLUTE
    ../../../../../../../middleware/lwip_2.0.0/src/api/netdb.c 0x00000000   Number         0  netdb.o ABSOLUTE
    ../../../../../../../middleware/lwip_2.0.0/src/api/netifapi.c 0x00000000   Number         0  netifapi.o ABSOLUTE
    ../../../../../../../middleware/lwip_2.0.0/src/api/sockets.c 0x00000000   Number         0  sockets.o ABSOLUTE
    ../../../../../../../middleware/lwip_2.0.0/src/api/tcpip.c 0x00000000   Number         0  tcpip.o ABSOLUTE
    ../../../../../../../middleware/lwip_2.0.0/src/core/def.c 0x00000000   Number         0  def.o ABSOLUTE
    ../../../../../../../middleware/lwip_2.0.0/src/core/dns.c 0x00000000   Number         0  dns.o ABSOLUTE
    ../../../../../../../middleware/lwip_2.0.0/src/core/inet_chksum.c 0x00000000   Number         0  inet_chksum.o ABSOLUTE
    ../../../../../../../middleware/lwip_2.0.0/src/core/init.c 0x00000000   Number         0  init.o ABSOLUTE
    ../../../../../../../middleware/lwip_2.0.0/src/core/ip.c 0x00000000   Number         0  ip.o ABSOLUTE
    ../../../../../../../middleware/lwip_2.0.0/src/core/ipv4/autoip.c 0x00000000   Number         0  autoip.o ABSOLUTE
    ../../../../../../../middleware/lwip_2.0.0/src/core/ipv4/dhcp.c 0x00000000   Number         0  dhcp.o ABSOLUTE
    ../../../../../../../middleware/lwip_2.0.0/src/core/ipv4/etharp.c 0x00000000   Number         0  etharp.o ABSOLUTE
    ../../../../../../../middleware/lwip_2.0.0/src/core/ipv4/icmp.c 0x00000000   Number         0  icmp.o ABSOLUTE
    ../../../../../../../middleware/lwip_2.0.0/src/core/ipv4/igmp.c 0x00000000   Number         0  igmp.o ABSOLUTE
    ../../../../../../../middleware/lwip_2.0.0/src/core/ipv4/ip4.c 0x00000000   Number         0  ip4.o ABSOLUTE
    ../../../../../../../middleware/lwip_2.0.0/src/core/ipv4/ip4_addr.c 0x00000000   Number         0  ip4_addr.o ABSOLUTE
    ../../../../../../../middleware/lwip_2.0.0/src/core/ipv4/ip4_frag.c 0x00000000   Number         0  ip4_frag.o ABSOLUTE
    ../../../../../../../middleware/lwip_2.0.0/src/core/ipv6/dhcp6.c 0x00000000   Number         0  dhcp6.o ABSOLUTE
    ../../../../../../../middleware/lwip_2.0.0/src/core/ipv6/ethip6.c 0x00000000   Number         0  ethip6.o ABSOLUTE
    ../../../../../../../middleware/lwip_2.0.0/src/core/ipv6/icmp6.c 0x00000000   Number         0  icmp6.o ABSOLUTE
    ../../../../../../../middleware/lwip_2.0.0/src/core/ipv6/inet6.c 0x00000000   Number         0  inet6.o ABSOLUTE
    ../../../../../../../middleware/lwip_2.0.0/src/core/ipv6/ip6.c 0x00000000   Number         0  ip6.o ABSOLUTE
    ../../../../../../../middleware/lwip_2.0.0/src/core/ipv6/ip6_addr.c 0x00000000   Number         0  ip6_addr.o ABSOLUTE
    ../../../../../../../middleware/lwip_2.0.0/src/core/ipv6/ip6_frag.c 0x00000000   Number         0  ip6_frag.o ABSOLUTE
    ../../../../../../../middleware/lwip_2.0.0/src/core/ipv6/mld6.c 0x00000000   Number         0  mld6.o ABSOLUTE
    ../../../../../../../middleware/lwip_2.0.0/src/core/ipv6/nd6.c 0x00000000   Number         0  nd6.o ABSOLUTE
    ../../../../../../../middleware/lwip_2.0.0/src/core/mem.c 0x00000000   Number         0  mem.o ABSOLUTE
    ../../../../../../../middleware/lwip_2.0.0/src/core/memp.c 0x00000000   Number         0  memp.o ABSOLUTE
    ../../../../../../../middleware/lwip_2.0.0/src/core/netif.c 0x00000000   Number         0  netif.o ABSOLUTE
    ../../../../../../../middleware/lwip_2.0.0/src/core/pbuf.c 0x00000000   Number         0  pbuf.o ABSOLUTE
    ../../../../../../../middleware/lwip_2.0.0/src/core/raw.c 0x00000000   Number         0  raw.o ABSOLUTE
    ../../../../../../../middleware/lwip_2.0.0/src/core/stats.c 0x00000000   Number         0  stats.o ABSOLUTE
    ../../../../../../../middleware/lwip_2.0.0/src/core/sys.c 0x00000000   Number         0  sys.o ABSOLUTE
    ../../../../../../../middleware/lwip_2.0.0/src/core/tcp.c 0x00000000   Number         0  tcp.o ABSOLUTE
    ../../../../../../../middleware/lwip_2.0.0/src/core/tcp_in.c 0x00000000   Number         0  tcp_in.o ABSOLUTE
    ../../../../../../../middleware/lwip_2.0.0/src/core/tcp_out.c 0x00000000   Number         0  tcp_out.o ABSOLUTE
    ../../../../../../../middleware/lwip_2.0.0/src/core/timeouts.c 0x00000000   Number         0  timeouts.o ABSOLUTE
    ../../../../../../../middleware/lwip_2.0.0/src/core/udp.c 0x00000000   Number         0  udp.o ABSOLUTE
    ../../../../../../../middleware/lwip_2.0.0/src/netif/ethernet.c 0x00000000   Number         0  ethernet.o ABSOLUTE
    ../../../../../../../middleware/lwip_2.0.0/src/netif/lowpan6.c 0x00000000   Number         0  lowpan6.o ABSOLUTE
    ../../../../../../../middleware/lwip_2.0.0/src/netif/ppp/auth.c 0x00000000   Number         0  auth.o ABSOLUTE
    ../../../../../../../middleware/lwip_2.0.0/src/netif/ppp/ccp.c 0x00000000   Number         0  ccp.o ABSOLUTE
    ../../../../../../../middleware/lwip_2.0.0/src/netif/ppp/chap-md5.c 0x00000000   Number         0  chap-md5.o ABSOLUTE
    ../../../../../../../middleware/lwip_2.0.0/src/netif/ppp/chap-new.c 0x00000000   Number         0  chap-new.o ABSOLUTE
    ../../../../../../../middleware/lwip_2.0.0/src/netif/ppp/chap_ms.c 0x00000000   Number         0  chap_ms.o ABSOLUTE
    ../../../../../../../middleware/lwip_2.0.0/src/netif/ppp/demand.c 0x00000000   Number         0  demand.o ABSOLUTE
    ../../../../../../../middleware/lwip_2.0.0/src/netif/ppp/eap.c 0x00000000   Number         0  eap.o ABSOLUTE
    ../../../../../../../middleware/lwip_2.0.0/src/netif/ppp/eui64.c 0x00000000   Number         0  eui64.o ABSOLUTE
    ../../../../../../../middleware/lwip_2.0.0/src/netif/ppp/fsm.c 0x00000000   Number         0  fsm.o ABSOLUTE
    ../../../../../../../middleware/lwip_2.0.0/src/netif/ppp/ipcp.c 0x00000000   Number         0  ipcp.o ABSOLUTE
    ../../../../../../../middleware/lwip_2.0.0/src/netif/ppp/ipv6cp.c 0x00000000   Number         0  ipv6cp.o ABSOLUTE
    ../../../../../../../middleware/lwip_2.0.0/src/netif/ppp/lcp.c 0x00000000   Number         0  lcp.o ABSOLUTE
    ../../../../../../../middleware/lwip_2.0.0/src/netif/ppp/lwip_ecp.c 0x00000000   Number         0  lwip_ecp.o ABSOLUTE
    ../../../../../../../middleware/lwip_2.0.0/src/netif/ppp/magic.c 0x00000000   Number         0  magic.o ABSOLUTE
    ../../../../../../../middleware/lwip_2.0.0/src/netif/ppp/mppe.c 0x00000000   Number         0  mppe.o ABSOLUTE
    ../../../../../../../middleware/lwip_2.0.0/src/netif/ppp/multilink.c 0x00000000   Number         0  multilink.o ABSOLUTE
    ../../../../../../../middleware/lwip_2.0.0/src/netif/ppp/ppp.c 0x00000000   Number         0  ppp.o ABSOLUTE
    ../../../../../../../middleware/lwip_2.0.0/src/netif/ppp/pppapi.c 0x00000000   Number         0  pppapi.o ABSOLUTE
    ../../../../../../../middleware/lwip_2.0.0/src/netif/ppp/pppcrypt.c 0x00000000   Number         0  pppcrypt.o ABSOLUTE
    ../../../../../../../middleware/lwip_2.0.0/src/netif/ppp/pppoe.c 0x00000000   Number         0  pppoe.o ABSOLUTE
    ../../../../../../../middleware/lwip_2.0.0/src/netif/ppp/pppol2tp.c 0x00000000   Number         0  pppol2tp.o ABSOLUTE
    ../../../../../../../middleware/lwip_2.0.0/src/netif/ppp/pppos.c 0x00000000   Number         0  pppos.o ABSOLUTE
    ../../../../../../../middleware/lwip_2.0.0/src/netif/ppp/upap.c 0x00000000   Number         0  upap.o ABSOLUTE
    ../../../../../../../middleware/lwip_2.0.0/src/netif/ppp/utils.c 0x00000000   Number         0  utils.o ABSOLUTE
    ../../../../../../../middleware/lwip_2.0.0/src/netif/ppp/vj.c 0x00000000   Number         0  vj.o ABSOLUTE
    ../../../../../../../middleware/lwip_2.0.0/src/netif/slipif.c 0x00000000   Number         0  slipif.o ABSOLUTE
    ../board.c                               0x00000000   Number         0  board.o ABSOLUTE
    ../clib/microlib/division.c              0x00000000   Number         0  uldiv.o ABSOLUTE
    ../clib/microlib/init/entry.s            0x00000000   Number         0  entry8a.o ABSOLUTE
    ../clib/microlib/init/entry.s            0x00000000   Number         0  entry4.o ABSOLUTE
    ../clib/microlib/init/entry.s            0x00000000   Number         0  entry.o ABSOLUTE
    ../clib/microlib/init/entry.s            0x00000000   Number         0  entry7b.o ABSOLUTE
    ../clib/microlib/init/entry.s            0x00000000   Number         0  entry10b.o ABSOLUTE
    ../clib/microlib/init/entry.s            0x00000000   Number         0  entry9a.o ABSOLUTE
    ../clib/microlib/init/entry.s            0x00000000   Number         0  entry11b.o ABSOLUTE
    ../clib/microlib/init/entry.s            0x00000000   Number         0  entry8b.o ABSOLUTE
    ../clib/microlib/init/entry.s            0x00000000   Number         0  entry10a.o ABSOLUTE
    ../clib/microlib/init/entry.s            0x00000000   Number         0  entry9b.o ABSOLUTE
    ../clib/microlib/init/entry.s            0x00000000   Number         0  entry7a.o ABSOLUTE
    ../clib/microlib/init/entry.s            0x00000000   Number         0  entry11a.o ABSOLUTE
    ../clib/microlib/init/entry.s            0x00000000   Number         0  entry5.o ABSOLUTE
    ../clib/microlib/longlong.c              0x00000000   Number         0  llushr.o ABSOLUTE
    ../clib/microlib/longlong.c              0x00000000   Number         0  llshl.o ABSOLUTE
    ../clib/microlib/string/memcmp.c         0x00000000   Number         0  memcmp.o ABSOLUTE
    ../clib/microlib/string/memcpy.c         0x00000000   Number         0  memcpya.o ABSOLUTE
    ../clib/microlib/string/memcpy.c         0x00000000   Number         0  memcpyb.o ABSOLUTE
    ../clib/microlib/string/memset.c         0x00000000   Number         0  memseta.o ABSOLUTE
    ../clib/microlib/string/strlen.c         0x00000000   Number         0  strlen.o ABSOLUTE
    ../clib/microlib/string/strncmp.c        0x00000000   Number         0  strncmp.o ABSOLUTE
    ../clock_config.c                        0x00000000   Number         0  clock_config.o ABSOLUTE
    ../fsl_phy.c                             0x00000000   Number         0  fsl_phy.o ABSOLUTE
    ../lwip_dhcp_bm.c                        0x00000000   Number         0  lwip_dhcp_bm.o ABSOLUTE
    ../pin_mux.c                             0x00000000   Number         0  pin_mux.o ABSOLUTE
    ..\..\..\..\..\..\..\devices\MK64F12\drivers\fsl_clock.c 0x00000000   Number         0  fsl_clock.o ABSOLUTE
    ..\..\..\..\..\..\..\devices\MK64F12\drivers\fsl_common.c 0x00000000   Number         0  fsl_common.o ABSOLUTE
    ..\..\..\..\..\..\..\devices\MK64F12\drivers\fsl_enet.c 0x00000000   Number         0  fsl_enet.o ABSOLUTE
    ..\..\..\..\..\..\..\devices\MK64F12\drivers\fsl_flash.c 0x00000000   Number         0  fsl_flash.o ABSOLUTE
    ..\..\..\..\..\..\..\devices\MK64F12\drivers\fsl_gpio.c 0x00000000   Number         0  fsl_gpio.o ABSOLUTE
    ..\..\..\..\..\..\..\devices\MK64F12\drivers\fsl_smc.c 0x00000000   Number         0  fsl_smc.o ABSOLUTE
    ..\..\..\..\..\..\..\devices\MK64F12\drivers\fsl_uart.c 0x00000000   Number         0  fsl_uart.o ABSOLUTE
    ..\..\..\..\..\..\..\devices\MK64F12\system_MK64F12.c 0x00000000   Number         0  system_mk64f12.o ABSOLUTE
    ..\..\..\..\..\..\..\devices\MK64F12\utilities\fsl_debug_console.c 0x00000000   Number         0  fsl_debug_console.o ABSOLUTE
    ..\..\..\..\..\..\..\middleware\lwip_2.0.0\port\ethernetif.c 0x00000000   Number         0  ethernetif.o ABSOLUTE
    ..\..\..\..\..\..\..\middleware\lwip_2.0.0\port\sys_arch.c 0x00000000   Number         0  sys_arch.o ABSOLUTE
    ..\..\..\..\..\..\..\middleware\lwip_2.0.0\src\api\api_lib.c 0x00000000   Number         0  api_lib.o ABSOLUTE
    ..\..\..\..\..\..\..\middleware\lwip_2.0.0\src\api\api_msg.c 0x00000000   Number         0  api_msg.o ABSOLUTE
    ..\..\..\..\..\..\..\middleware\lwip_2.0.0\src\api\err.c 0x00000000   Number         0  err.o ABSOLUTE
    ..\..\..\..\..\..\..\middleware\lwip_2.0.0\src\api\netbuf.c 0x00000000   Number         0  netbuf.o ABSOLUTE
    ..\..\..\..\..\..\..\middleware\lwip_2.0.0\src\api\netdb.c 0x00000000   Number         0  netdb.o ABSOLUTE
    ..\..\..\..\..\..\..\middleware\lwip_2.0.0\src\api\netifapi.c 0x00000000   Number         0  netifapi.o ABSOLUTE
    ..\..\..\..\..\..\..\middleware\lwip_2.0.0\src\api\sockets.c 0x00000000   Number         0  sockets.o ABSOLUTE
    ..\..\..\..\..\..\..\middleware\lwip_2.0.0\src\api\tcpip.c 0x00000000   Number         0  tcpip.o ABSOLUTE
    ..\..\..\..\..\..\..\middleware\lwip_2.0.0\src\core\def.c 0x00000000   Number         0  def.o ABSOLUTE
    ..\..\..\..\..\..\..\middleware\lwip_2.0.0\src\core\dns.c 0x00000000   Number         0  dns.o ABSOLUTE
    ..\..\..\..\..\..\..\middleware\lwip_2.0.0\src\core\inet_chksum.c 0x00000000   Number         0  inet_chksum.o ABSOLUTE
    ..\..\..\..\..\..\..\middleware\lwip_2.0.0\src\core\init.c 0x00000000   Number         0  init.o ABSOLUTE
    ..\..\..\..\..\..\..\middleware\lwip_2.0.0\src\core\ip.c 0x00000000   Number         0  ip.o ABSOLUTE
    ..\..\..\..\..\..\..\middleware\lwip_2.0.0\src\core\ipv4\autoip.c 0x00000000   Number         0  autoip.o ABSOLUTE
    ..\..\..\..\..\..\..\middleware\lwip_2.0.0\src\core\ipv4\dhcp.c 0x00000000   Number         0  dhcp.o ABSOLUTE
    ..\..\..\..\..\..\..\middleware\lwip_2.0.0\src\core\ipv4\etharp.c 0x00000000   Number         0  etharp.o ABSOLUTE
    ..\..\..\..\..\..\..\middleware\lwip_2.0.0\src\core\ipv4\icmp.c 0x00000000   Number         0  icmp.o ABSOLUTE
    ..\..\..\..\..\..\..\middleware\lwip_2.0.0\src\core\ipv4\igmp.c 0x00000000   Number         0  igmp.o ABSOLUTE
    ..\..\..\..\..\..\..\middleware\lwip_2.0.0\src\core\ipv4\ip4.c 0x00000000   Number         0  ip4.o ABSOLUTE
    ..\..\..\..\..\..\..\middleware\lwip_2.0.0\src\core\ipv4\ip4_addr.c 0x00000000   Number         0  ip4_addr.o ABSOLUTE
    ..\..\..\..\..\..\..\middleware\lwip_2.0.0\src\core\ipv4\ip4_frag.c 0x00000000   Number         0  ip4_frag.o ABSOLUTE
    ..\..\..\..\..\..\..\middleware\lwip_2.0.0\src\core\ipv6\dhcp6.c 0x00000000   Number         0  dhcp6.o ABSOLUTE
    ..\..\..\..\..\..\..\middleware\lwip_2.0.0\src\core\ipv6\ethip6.c 0x00000000   Number         0  ethip6.o ABSOLUTE
    ..\..\..\..\..\..\..\middleware\lwip_2.0.0\src\core\ipv6\icmp6.c 0x00000000   Number         0  icmp6.o ABSOLUTE
    ..\..\..\..\..\..\..\middleware\lwip_2.0.0\src\core\ipv6\inet6.c 0x00000000   Number         0  inet6.o ABSOLUTE
    ..\..\..\..\..\..\..\middleware\lwip_2.0.0\src\core\ipv6\ip6.c 0x00000000   Number         0  ip6.o ABSOLUTE
    ..\..\..\..\..\..\..\middleware\lwip_2.0.0\src\core\ipv6\ip6_addr.c 0x00000000   Number         0  ip6_addr.o ABSOLUTE
    ..\..\..\..\..\..\..\middleware\lwip_2.0.0\src\core\ipv6\ip6_frag.c 0x00000000   Number         0  ip6_frag.o ABSOLUTE
    ..\..\..\..\..\..\..\middleware\lwip_2.0.0\src\core\ipv6\mld6.c 0x00000000   Number         0  mld6.o ABSOLUTE
    ..\..\..\..\..\..\..\middleware\lwip_2.0.0\src\core\ipv6\nd6.c 0x00000000   Number         0  nd6.o ABSOLUTE
    ..\..\..\..\..\..\..\middleware\lwip_2.0.0\src\core\mem.c 0x00000000   Number         0  mem.o ABSOLUTE
    ..\..\..\..\..\..\..\middleware\lwip_2.0.0\src\core\memp.c 0x00000000   Number         0  memp.o ABSOLUTE
    ..\..\..\..\..\..\..\middleware\lwip_2.0.0\src\core\netif.c 0x00000000   Number         0  netif.o ABSOLUTE
    ..\..\..\..\..\..\..\middleware\lwip_2.0.0\src\core\pbuf.c 0x00000000   Number         0  pbuf.o ABSOLUTE
    ..\..\..\..\..\..\..\middleware\lwip_2.0.0\src\core\raw.c 0x00000000   Number         0  raw.o ABSOLUTE
    ..\..\..\..\..\..\..\middleware\lwip_2.0.0\src\core\stats.c 0x00000000   Number         0  stats.o ABSOLUTE
    ..\..\..\..\..\..\..\middleware\lwip_2.0.0\src\core\sys.c 0x00000000   Number         0  sys.o ABSOLUTE
    ..\..\..\..\..\..\..\middleware\lwip_2.0.0\src\core\tcp.c 0x00000000   Number         0  tcp.o ABSOLUTE
    ..\..\..\..\..\..\..\middleware\lwip_2.0.0\src\core\tcp_in.c 0x00000000   Number         0  tcp_in.o ABSOLUTE
    ..\..\..\..\..\..\..\middleware\lwip_2.0.0\src\core\tcp_out.c 0x00000000   Number         0  tcp_out.o ABSOLUTE
    ..\..\..\..\..\..\..\middleware\lwip_2.0.0\src\core\timeouts.c 0x00000000   Number         0  timeouts.o ABSOLUTE
    ..\..\..\..\..\..\..\middleware\lwip_2.0.0\src\core\udp.c 0x00000000   Number         0  udp.o ABSOLUTE
    ..\..\..\..\..\..\..\middleware\lwip_2.0.0\src\netif\ethernet.c 0x00000000   Number         0  ethernet.o ABSOLUTE
    ..\..\..\..\..\..\..\middleware\lwip_2.0.0\src\netif\lowpan6.c 0x00000000   Number         0  lowpan6.o ABSOLUTE
    ..\..\..\..\..\..\..\middleware\lwip_2.0.0\src\netif\ppp\auth.c 0x00000000   Number         0  auth.o ABSOLUTE
    ..\..\..\..\..\..\..\middleware\lwip_2.0.0\src\netif\ppp\ccp.c 0x00000000   Number         0  ccp.o ABSOLUTE
    ..\..\..\..\..\..\..\middleware\lwip_2.0.0\src\netif\ppp\chap-md5.c 0x00000000   Number         0  chap-md5.o ABSOLUTE
    ..\..\..\..\..\..\..\middleware\lwip_2.0.0\src\netif\ppp\chap-new.c 0x00000000   Number         0  chap-new.o ABSOLUTE
    ..\..\..\..\..\..\..\middleware\lwip_2.0.0\src\netif\ppp\chap_ms.c 0x00000000   Number         0  chap_ms.o ABSOLUTE
    ..\..\..\..\..\..\..\middleware\lwip_2.0.0\src\netif\ppp\demand.c 0x00000000   Number         0  demand.o ABSOLUTE
    ..\..\..\..\..\..\..\middleware\lwip_2.0.0\src\netif\ppp\eap.c 0x00000000   Number         0  eap.o ABSOLUTE
    ..\..\..\..\..\..\..\middleware\lwip_2.0.0\src\netif\ppp\eui64.c 0x00000000   Number         0  eui64.o ABSOLUTE
    ..\..\..\..\..\..\..\middleware\lwip_2.0.0\src\netif\ppp\fsm.c 0x00000000   Number         0  fsm.o ABSOLUTE
    ..\..\..\..\..\..\..\middleware\lwip_2.0.0\src\netif\ppp\ipcp.c 0x00000000   Number         0  ipcp.o ABSOLUTE
    ..\..\..\..\..\..\..\middleware\lwip_2.0.0\src\netif\ppp\ipv6cp.c 0x00000000   Number         0  ipv6cp.o ABSOLUTE
    ..\..\..\..\..\..\..\middleware\lwip_2.0.0\src\netif\ppp\lcp.c 0x00000000   Number         0  lcp.o ABSOLUTE
    ..\..\..\..\..\..\..\middleware\lwip_2.0.0\src\netif\ppp\lwip_ecp.c 0x00000000   Number         0  lwip_ecp.o ABSOLUTE
    ..\..\..\..\..\..\..\middleware\lwip_2.0.0\src\netif\ppp\magic.c 0x00000000   Number         0  magic.o ABSOLUTE
    ..\..\..\..\..\..\..\middleware\lwip_2.0.0\src\netif\ppp\mppe.c 0x00000000   Number         0  mppe.o ABSOLUTE
    ..\..\..\..\..\..\..\middleware\lwip_2.0.0\src\netif\ppp\multilink.c 0x00000000   Number         0  multilink.o ABSOLUTE
    ..\..\..\..\..\..\..\middleware\lwip_2.0.0\src\netif\ppp\ppp.c 0x00000000   Number         0  ppp.o ABSOLUTE
    ..\..\..\..\..\..\..\middleware\lwip_2.0.0\src\netif\ppp\pppapi.c 0x00000000   Number         0  pppapi.o ABSOLUTE
    ..\..\..\..\..\..\..\middleware\lwip_2.0.0\src\netif\ppp\pppcrypt.c 0x00000000   Number         0  pppcrypt.o ABSOLUTE
    ..\..\..\..\..\..\..\middleware\lwip_2.0.0\src\netif\ppp\pppoe.c 0x00000000   Number         0  pppoe.o ABSOLUTE
    ..\..\..\..\..\..\..\middleware\lwip_2.0.0\src\netif\ppp\pppol2tp.c 0x00000000   Number         0  pppol2tp.o ABSOLUTE
    ..\..\..\..\..\..\..\middleware\lwip_2.0.0\src\netif\ppp\pppos.c 0x00000000   Number         0  pppos.o ABSOLUTE
    ..\..\..\..\..\..\..\middleware\lwip_2.0.0\src\netif\ppp\upap.c 0x00000000   Number         0  upap.o ABSOLUTE
    ..\..\..\..\..\..\..\middleware\lwip_2.0.0\src\netif\ppp\utils.c 0x00000000   Number         0  utils.o ABSOLUTE
    ..\..\..\..\..\..\..\middleware\lwip_2.0.0\src\netif\ppp\vj.c 0x00000000   Number         0  vj.o ABSOLUTE
    ..\..\..\..\..\..\..\middleware\lwip_2.0.0\src\netif\slipif.c 0x00000000   Number         0  slipif.o ABSOLUTE
    ..\board.c                               0x00000000   Number         0  board.o ABSOLUTE
    ..\clock_config.c                        0x00000000   Number         0  clock_config.o ABSOLUTE
    ..\fsl_phy.c                             0x00000000   Number         0  fsl_phy.o ABSOLUTE
    ..\lwip_dhcp_bm.c                        0x00000000   Number         0  lwip_dhcp_bm.o ABSOLUTE
    ..\pin_mux.c                             0x00000000   Number         0  pin_mux.o ABSOLUTE
    dc.s                                     0x00000000   Number         0  dc.o ABSOLUTE
    handlers.s                               0x00000000   Number         0  handlers.o ABSOLUTE
    init.s                                   0x00000000   Number         0  init.o ABSOLUTE
    FlashConfig                              0x00000400   Section       16  startup_mk64f12.o(FlashConfig)
    .ARM.Collect$$$$00000000                 0x00000410   Section        0  entry.o(.ARM.Collect$$$$00000000)
    .ARM.Collect$$$$00000003                 0x00000410   Section        4  entry4.o(.ARM.Collect$$$$00000003)
    .ARM.Collect$$$$00000004                 0x00000414   Section        4  entry5.o(.ARM.Collect$$$$00000004)
    .ARM.Collect$$$$00000008                 0x00000418   Section        0  entry7b.o(.ARM.Collect$$$$00000008)
    .ARM.Collect$$$$0000000A                 0x00000418   Section        0  entry8b.o(.ARM.Collect$$$$0000000A)
    .ARM.Collect$$$$0000000B                 0x00000418   Section        8  entry9a.o(.ARM.Collect$$$$0000000B)
    .ARM.Collect$$$$0000000D                 0x00000420   Section        0  entry10a.o(.ARM.Collect$$$$0000000D)
    .ARM.Collect$$$$0000000F                 0x00000420   Section        0  entry11a.o(.ARM.Collect$$$$0000000F)
    .ARM.Collect$$$$00002714                 0x00000420   Section        4  entry4.o(.ARM.Collect$$$$00002714)
    __lit__00000000                          0x00000420   Data           4  entry4.o(.ARM.Collect$$$$00002714)
    .text                                    0x00000424   Section      452  startup_mk64f12.o(.text)
    $v0                                      0x00000424   Number         0  startup_mk64f12.o(.text)
    .text                                    0x000005e8   Section        0  uldiv.o(.text)
    .text                                    0x0000064a   Section        0  memcpya.o(.text)
    .text                                    0x0000066e   Section        0  memseta.o(.text)
    .text                                    0x00000692   Section        0  strlen.o(.text)
    .text                                    0x000006a0   Section        0  memcmp.o(.text)
    .text                                    0x000006ba   Section        0  llshl.o(.text)
    .text                                    0x000006d8   Section        0  llushr.o(.text)
    .text                                    0x000006f8   Section       36  init.o(.text)
    i.BOARD_BootClockRUN                     0x0000071c   Section        0  clock_config.o(i.BOARD_BootClockRUN)
    i.BOARD_InitDebugConsole                 0x00000788   Section        0  board.o(i.BOARD_InitDebugConsole)
    i.BOARD_InitPins                         0x000007a4   Section        0  pin_mux.o(i.BOARD_InitPins)
    i.CLOCK_BootToPeeMode                    0x00000890   Section        0  fsl_clock.o(i.CLOCK_BootToPeeMode)
    i.CLOCK_CONFIG_SetFllExtRefDiv           0x0000091c   Section        0  clock_config.o(i.CLOCK_CONFIG_SetFllExtRefDiv)
    CLOCK_CONFIG_SetFllExtRefDiv             0x0000091d   Thumb Code    14  clock_config.o(i.CLOCK_CONFIG_SetFllExtRefDiv)
    i.CLOCK_EnableClock                      0x00000930   Section        0  pin_mux.o(i.CLOCK_EnableClock)
    CLOCK_EnableClock                        0x00000931   Thumb Code    18  pin_mux.o(i.CLOCK_EnableClock)
    i.CLOCK_EnablePll0                       0x00000948   Section        0  fsl_clock.o(i.CLOCK_EnablePll0)
    i.CLOCK_GetCoreSysClkFreq                0x000009e0   Section        0  fsl_clock.o(i.CLOCK_GetCoreSysClkFreq)
    i.CLOCK_GetEr32kClkFreq                  0x000009fc   Section        0  fsl_clock.o(i.CLOCK_GetEr32kClkFreq)
    i.CLOCK_GetFixedFreqClkFreq              0x00000aa8   Section        0  fsl_clock.o(i.CLOCK_GetFixedFreqClkFreq)
    i.CLOCK_GetFllExtRefClkFreq              0x00000ac4   Section        0  fsl_clock.o(i.CLOCK_GetFllExtRefClkFreq)
    CLOCK_GetFllExtRefClkFreq                0x00000ac5   Thumb Code   108  fsl_clock.o(i.CLOCK_GetFllExtRefClkFreq)
    i.CLOCK_GetFllFreq                       0x00000b34   Section        0  fsl_clock.o(i.CLOCK_GetFllFreq)
    i.CLOCK_GetFllRefClkFreq                 0x00000b80   Section        0  fsl_clock.o(i.CLOCK_GetFllRefClkFreq)
    CLOCK_GetFllRefClkFreq                   0x00000b81   Thumb Code    24  fsl_clock.o(i.CLOCK_GetFllRefClkFreq)
    i.CLOCK_GetFreq                          0x00000ba0   Section        0  fsl_clock.o(i.CLOCK_GetFreq)
    i.CLOCK_GetInternalRefClkFreq            0x00000c68   Section        0  fsl_clock.o(i.CLOCK_GetInternalRefClkFreq)
    i.CLOCK_GetInternalRefClkSelectFreq      0x00000c84   Section        0  fsl_clock.o(i.CLOCK_GetInternalRefClkSelectFreq)
    CLOCK_GetInternalRefClkSelectFreq        0x00000c85   Thumb Code    32  fsl_clock.o(i.CLOCK_GetInternalRefClkSelectFreq)
    i.CLOCK_GetMcgExtClkFreq                 0x00000cb0   Section        0  fsl_clock.o(i.CLOCK_GetMcgExtClkFreq)
    CLOCK_GetMcgExtClkFreq                   0x00000cb1   Thumb Code    84  fsl_clock.o(i.CLOCK_GetMcgExtClkFreq)
    i.CLOCK_GetOsc0ErClkFreq                 0x00000d6c   Section        0  fsl_clock.o(i.CLOCK_GetOsc0ErClkFreq)
    i.CLOCK_GetOscRangeFromFreq              0x00000de8   Section        0  fsl_clock.o(i.CLOCK_GetOscRangeFromFreq)
    CLOCK_GetOscRangeFromFreq                0x00000de9   Thumb Code    28  fsl_clock.o(i.CLOCK_GetOscRangeFromFreq)
    i.CLOCK_GetOutClkFreq                    0x00000e08   Section        0  fsl_clock.o(i.CLOCK_GetOutClkFreq)
    i.CLOCK_GetPll0Freq                      0x00000e44   Section        0  fsl_clock.o(i.CLOCK_GetPll0Freq)
    i.CLOCK_GetPll0RefFreq                   0x00000ed4   Section        0  fsl_clock.o(i.CLOCK_GetPll0RefFreq)
    CLOCK_GetPll0RefFreq                     0x00000ed5   Thumb Code     8  fsl_clock.o(i.CLOCK_GetPll0RefFreq)
    i.CLOCK_GetPllFllSelClkFreq              0x00000edc   Section        0  fsl_clock.o(i.CLOCK_GetPllFllSelClkFreq)
    i.CLOCK_InitOsc0                         0x00000f14   Section        0  fsl_clock.o(i.CLOCK_InitOsc0)
    i.CLOCK_SetExternalRefClkConfig          0x00000f80   Section        0  fsl_clock.o(i.CLOCK_SetExternalRefClkConfig)
    i.CLOCK_SetInternalRefClkConfig          0x00000fbc   Section        0  fsl_clock.o(i.CLOCK_SetInternalRefClkConfig)
    i.CLOCK_SetPbeMode                       0x00001054   Section        0  fsl_clock.o(i.CLOCK_SetPbeMode)
    i.CLOCK_SetSimConfig                     0x00001118   Section        0  fsl_clock.o(i.CLOCK_SetSimConfig)
    i.DbgConsole_ConvertRadixNumToString     0x00001148   Section        0  fsl_debug_console.o(i.DbgConsole_ConvertRadixNumToString)
    DbgConsole_ConvertRadixNumToString       0x00001149   Thumb Code   168  fsl_debug_console.o(i.DbgConsole_ConvertRadixNumToString)
    i.DbgConsole_Init                        0x000011f0   Section        0  fsl_debug_console.o(i.DbgConsole_Init)
    i.DbgConsole_Printf                      0x00001288   Section        0  fsl_debug_console.o(i.DbgConsole_Printf)
    i.DbgConsole_PrintfFormattedData         0x000012bc   Section        0  fsl_debug_console.o(i.DbgConsole_PrintfFormattedData)
    DbgConsole_PrintfFormattedData           0x000012bd   Thumb Code   570  fsl_debug_console.o(i.DbgConsole_PrintfFormattedData)
    i.DbgConsole_PrintfPaddingCharacter      0x000014f6   Section        0  fsl_debug_console.o(i.DbgConsole_PrintfPaddingCharacter)
    DbgConsole_PrintfPaddingCharacter        0x000014f7   Thumb Code    40  fsl_debug_console.o(i.DbgConsole_PrintfPaddingCharacter)
    i.DbgConsole_Putchar                     0x00001520   Section        0  fsl_debug_console.o(i.DbgConsole_Putchar)
    i.ENET_1588_Timer_IRQHandler             0x00001544   Section        0  fsl_enet.o(i.ENET_1588_Timer_IRQHandler)
    i.ENET_ClearInterruptStatus              0x00001560   Section        0  fsl_phy.o(i.ENET_ClearInterruptStatus)
    ENET_ClearInterruptStatus                0x00001561   Thumb Code     4  fsl_phy.o(i.ENET_ClearInterruptStatus)
    i.ENET_ErrorIRQHandler                   0x00001564   Section        0  fsl_enet.o(i.ENET_ErrorIRQHandler)
    i.ENET_Error_IRQHandler                  0x00001614   Section        0  fsl_enet.o(i.ENET_Error_IRQHandler)
    i.ENET_GetDefaultConfig                  0x00001630   Section        0  fsl_enet.o(i.ENET_GetDefaultConfig)
    i.ENET_GetInstance                       0x0000169c   Section        0  fsl_enet.o(i.ENET_GetInstance)
    i.ENET_GetRxFrameSize                    0x0000172c   Section        0  fsl_enet.o(i.ENET_GetRxFrameSize)
    i.ENET_Init                              0x00001818   Section        0  fsl_enet.o(i.ENET_Init)
    i.ENET_ReadFrame                         0x00001ac8   Section        0  fsl_enet.o(i.ENET_ReadFrame)
    i.ENET_ReceiveIRQHandler                 0x00001bec   Section        0  fsl_enet.o(i.ENET_ReceiveIRQHandler)
    i.ENET_Receive_IRQHandler                0x00001c68   Section        0  fsl_enet.o(i.ENET_Receive_IRQHandler)
    i.ENET_SendFrame                         0x00001c84   Section        0  fsl_enet.o(i.ENET_SendFrame)
    i.ENET_SetHandler                        0x00001e30   Section        0  fsl_enet.o(i.ENET_SetHandler)
    ENET_SetHandler                          0x00001e31   Thumb Code   128  fsl_enet.o(i.ENET_SetHandler)
    i.ENET_SetMacAddr                        0x00001edc   Section        0  fsl_enet.o(i.ENET_SetMacAddr)
    i.ENET_SetMacController                  0x00001f08   Section        0  fsl_enet.o(i.ENET_SetMacController)
    ENET_SetMacController                    0x00001f09   Thumb Code   428  fsl_enet.o(i.ENET_SetMacController)
    i.ENET_SetRxBufferDescriptors            0x000020b8   Section        0  fsl_enet.o(i.ENET_SetRxBufferDescriptors)
    ENET_SetRxBufferDescriptors              0x000020b9   Thumb Code   100  fsl_enet.o(i.ENET_SetRxBufferDescriptors)
    i.ENET_SetSMI                            0x00002178   Section        0  fsl_enet.o(i.ENET_SetSMI)
    i.ENET_SetTxBufferDescriptors            0x00002220   Section        0  fsl_enet.o(i.ENET_SetTxBufferDescriptors)
    ENET_SetTxBufferDescriptors              0x00002221   Thumb Code    94  fsl_enet.o(i.ENET_SetTxBufferDescriptors)
    i.ENET_StartSMIRead                      0x000022dc   Section        0  fsl_enet.o(i.ENET_StartSMIRead)
    i.ENET_StartSMIWrite                     0x00002308   Section        0  fsl_enet.o(i.ENET_StartSMIWrite)
    i.ENET_TransmitIRQHandler                0x0000233c   Section        0  fsl_enet.o(i.ENET_TransmitIRQHandler)
    i.ENET_Transmit_IRQHandler               0x000023b8   Section        0  fsl_enet.o(i.ENET_Transmit_IRQHandler)
    i.ENET_UpdateReadBuffers                 0x000023d4   Section        0  fsl_enet.o(i.ENET_UpdateReadBuffers)
    ENET_UpdateReadBuffers                   0x000023d5   Thumb Code    76  fsl_enet.o(i.ENET_UpdateReadBuffers)
    i.EnableIRQ                              0x00002460   Section        0  fsl_enet.o(i.EnableIRQ)
    EnableIRQ                                0x00002461   Thumb Code    36  fsl_enet.o(i.EnableIRQ)
    i.PHY_GetLinkSpeedDuplex                 0x00002484   Section        0  fsl_phy.o(i.PHY_GetLinkSpeedDuplex)
    i.PHY_GetLinkStatus                      0x00002500   Section        0  fsl_phy.o(i.PHY_GetLinkStatus)
    i.PHY_Init                               0x00002558   Section        0  fsl_phy.o(i.PHY_Init)
    i.PHY_Read                               0x0000262c   Section        0  fsl_phy.o(i.PHY_Read)
    i.PHY_Write                              0x000026b0   Section        0  fsl_phy.o(i.PHY_Write)
    i.PORT_SetPinConfig                      0x00002708   Section        0  pin_mux.o(i.PORT_SetPinConfig)
    PORT_SetPinConfig                        0x00002709   Thumb Code    38  pin_mux.o(i.PORT_SetPinConfig)
    i.PORT_SetPinMux                         0x00002770   Section        0  pin_mux.o(i.PORT_SetPinMux)
    PORT_SetPinMux                           0x00002771   Thumb Code    14  pin_mux.o(i.PORT_SetPinMux)
    i.SysTick_Handler                        0x0000277e   Section        0  lwip_dhcp_bm.o(i.SysTick_Handler)
    i.SystemInit                             0x00002788   Section        0  system_mk64f12.o(i.SystemInit)
    i.UART0_DriverIRQHandler                 0x000027b4   Section        0  fsl_uart.o(i.UART0_DriverIRQHandler)
    i.UART0_RX_TX_DriverIRQHandler           0x000027d0   Section        0  fsl_uart.o(i.UART0_RX_TX_DriverIRQHandler)
    i.UART1_DriverIRQHandler                 0x000027d8   Section        0  fsl_uart.o(i.UART1_DriverIRQHandler)
    i.UART1_RX_TX_DriverIRQHandler           0x000027f4   Section        0  fsl_uart.o(i.UART1_RX_TX_DriverIRQHandler)
    i.UART2_DriverIRQHandler                 0x000027fc   Section        0  fsl_uart.o(i.UART2_DriverIRQHandler)
    i.UART2_RX_TX_DriverIRQHandler           0x00002818   Section        0  fsl_uart.o(i.UART2_RX_TX_DriverIRQHandler)
    i.UART3_DriverIRQHandler                 0x00002820   Section        0  fsl_uart.o(i.UART3_DriverIRQHandler)
    i.UART3_RX_TX_DriverIRQHandler           0x0000283c   Section        0  fsl_uart.o(i.UART3_RX_TX_DriverIRQHandler)
    i.UART4_DriverIRQHandler                 0x00002844   Section        0  fsl_uart.o(i.UART4_DriverIRQHandler)
    i.UART4_RX_TX_DriverIRQHandler           0x00002860   Section        0  fsl_uart.o(i.UART4_RX_TX_DriverIRQHandler)
    i.UART5_DriverIRQHandler                 0x00002868   Section        0  fsl_uart.o(i.UART5_DriverIRQHandler)
    i.UART5_RX_TX_DriverIRQHandler           0x00002884   Section        0  fsl_uart.o(i.UART5_RX_TX_DriverIRQHandler)
    i.UART_GetDefaultConfig                  0x0000288c   Section        0  fsl_uart.o(i.UART_GetDefaultConfig)
    i.UART_GetInstance                       0x000028fc   Section        0  fsl_uart.o(i.UART_GetInstance)
    i.UART_GetStatusFlags                    0x00002988   Section        0  fsl_uart.o(i.UART_GetStatusFlags)
    i.UART_Init                              0x000029a0   Section        0  fsl_uart.o(i.UART_Init)
    i.UART_ReadBlocking                      0x00002c44   Section        0  fsl_uart.o(i.UART_ReadBlocking)
    i.UART_WriteBlocking                     0x00002cf4   Section        0  fsl_uart.o(i.UART_WriteBlocking)
    i.__aeabi_assert                         0x00002d14   Section        0  fsl_common.o(i.__aeabi_assert)
    i.__scatterload_copy                     0x00002d58   Section       14  handlers.o(i.__scatterload_copy)
    i.__scatterload_null                     0x00002d66   Section        2  handlers.o(i.__scatterload_null)
    i.__scatterload_zeroinit                 0x00002d68   Section       14  handlers.o(i.__scatterload_zeroinit)
    i.cyclic_timer                           0x00002d78   Section        0  timeouts.o(i.cyclic_timer)
    cyclic_timer                             0x00002d79   Thumb Code    22  timeouts.o(i.cyclic_timer)
    i.dhcp_arp_reply                         0x00002d94   Section        0  dhcp.o(i.dhcp_arp_reply)
    i.dhcp_bind                              0x00002de0   Section        0  dhcp.o(i.dhcp_bind)
    dhcp_bind                                0x00002de1   Thumb Code   302  dhcp.o(i.dhcp_bind)
    i.dhcp_check                             0x00002f44   Section        0  dhcp.o(i.dhcp_check)
    dhcp_check                               0x00002f45   Thumb Code    76  dhcp.o(i.dhcp_check)
    i.dhcp_coarse_tmr                        0x00002f90   Section        0  dhcp.o(i.dhcp_coarse_tmr)
    i.dhcp_create_msg                        0x00003008   Section        0  dhcp.o(i.dhcp_create_msg)
    dhcp_create_msg                          0x00003009   Thumb Code   386  dhcp.o(i.dhcp_create_msg)
    i.dhcp_dec_pcb_refcount                  0x00003264   Section        0  dhcp.o(i.dhcp_dec_pcb_refcount)
    dhcp_dec_pcb_refcount                    0x00003265   Thumb Code    52  dhcp.o(i.dhcp_dec_pcb_refcount)
    i.dhcp_decline                           0x000032c4   Section        0  dhcp.o(i.dhcp_decline)
    dhcp_decline                             0x000032c5   Thumb Code   154  dhcp.o(i.dhcp_decline)
    i.dhcp_delete_msg                        0x0000336c   Section        0  dhcp.o(i.dhcp_delete_msg)
    dhcp_delete_msg                          0x0000336d   Thumb Code    66  dhcp.o(i.dhcp_delete_msg)
    i.dhcp_discover                          0x00003420   Section        0  dhcp.o(i.dhcp_discover)
    dhcp_discover                            0x00003421   Thumb Code   228  dhcp.o(i.dhcp_discover)
    i.dhcp_fine_tmr                          0x00003514   Section        0  dhcp.o(i.dhcp_fine_tmr)
    i.dhcp_handle_ack                        0x00003554   Section        0  dhcp.o(i.dhcp_handle_ack)
    dhcp_handle_ack                          0x00003555   Thumb Code   118  dhcp.o(i.dhcp_handle_ack)
    i.dhcp_handle_nak                        0x000035d4   Section        0  dhcp.o(i.dhcp_handle_nak)
    dhcp_handle_nak                          0x000035d5   Thumb Code    38  dhcp.o(i.dhcp_handle_nak)
    i.dhcp_handle_offer                      0x00003600   Section        0  dhcp.o(i.dhcp_handle_offer)
    dhcp_handle_offer                        0x00003601   Thumb Code    54  dhcp.o(i.dhcp_handle_offer)
    i.dhcp_inc_pcb_refcount                  0x00003640   Section        0  dhcp.o(i.dhcp_inc_pcb_refcount)
    dhcp_inc_pcb_refcount                    0x00003641   Thumb Code   112  dhcp.o(i.dhcp_inc_pcb_refcount)
    i.dhcp_option                            0x000036e8   Section        0  dhcp.o(i.dhcp_option)
    dhcp_option                              0x000036e9   Thumb Code    54  dhcp.o(i.dhcp_option)
    i.dhcp_option_byte                       0x00003724   Section        0  dhcp.o(i.dhcp_option_byte)
    dhcp_option_byte                         0x00003725   Thumb Code    36  dhcp.o(i.dhcp_option_byte)
    i.dhcp_option_long                       0x00003784   Section        0  dhcp.o(i.dhcp_option_long)
    dhcp_option_long                         0x00003785   Thumb Code    84  dhcp.o(i.dhcp_option_long)
    i.dhcp_option_short                      0x00003818   Section        0  dhcp.o(i.dhcp_option_short)
    dhcp_option_short                        0x00003819   Thumb Code    52  dhcp.o(i.dhcp_option_short)
    i.dhcp_option_trailer                    0x00003850   Section        0  dhcp.o(i.dhcp_option_trailer)
    dhcp_option_trailer                      0x00003851   Thumb Code   102  dhcp.o(i.dhcp_option_trailer)
    i.dhcp_parse_reply                       0x00003948   Section        0  dhcp.o(i.dhcp_parse_reply)
    dhcp_parse_reply                         0x00003949   Thumb Code   912  dhcp.o(i.dhcp_parse_reply)
    i.dhcp_rebind                            0x00003d70   Section        0  dhcp.o(i.dhcp_rebind)
    dhcp_rebind                              0x00003d71   Thumb Code   196  dhcp.o(i.dhcp_rebind)
    i.dhcp_reboot                            0x00003e40   Section        0  dhcp.o(i.dhcp_reboot)
    dhcp_reboot                              0x00003e41   Thumb Code   224  dhcp.o(i.dhcp_reboot)
    i.dhcp_recv                              0x00003f2c   Section        0  dhcp.o(i.dhcp_recv)
    dhcp_recv                                0x00003f2d   Thumb Code   356  dhcp.o(i.dhcp_recv)
    i.dhcp_release                           0x000040b0   Section        0  dhcp.o(i.dhcp_release)
    i.dhcp_renew                             0x00004168   Section        0  dhcp.o(i.dhcp_renew)
    i.dhcp_select                            0x00004238   Section        0  dhcp.o(i.dhcp_select)
    dhcp_select                              0x00004239   Thumb Code   258  dhcp.o(i.dhcp_select)
    i.dhcp_set_state                         0x0000434c   Section        0  dhcp.o(i.dhcp_set_state)
    dhcp_set_state                           0x0000434d   Thumb Code    16  dhcp.o(i.dhcp_set_state)
    i.dhcp_start                             0x0000435c   Section        0  dhcp.o(i.dhcp_start)
    i.dhcp_stop                              0x00004484   Section        0  dhcp.o(i.dhcp_stop)
    i.dhcp_supplied_address                  0x000044f4   Section        0  dhcp.o(i.dhcp_supplied_address)
    i.dhcp_t1_timeout                        0x00004516   Section        0  dhcp.o(i.dhcp_t1_timeout)
    dhcp_t1_timeout                          0x00004517   Thumb Code    74  dhcp.o(i.dhcp_t1_timeout)
    i.dhcp_t2_timeout                        0x00004560   Section        0  dhcp.o(i.dhcp_t2_timeout)
    dhcp_t2_timeout                          0x00004561   Thumb Code    80  dhcp.o(i.dhcp_t2_timeout)
    i.dhcp_timeout                           0x000045b0   Section        0  dhcp.o(i.dhcp_timeout)
    dhcp_timeout                             0x000045b1   Thumb Code   136  dhcp.o(i.dhcp_timeout)
    i.do_memp_free_pool                      0x00004638   Section        0  memp.o(i.do_memp_free_pool)
    do_memp_free_pool                        0x00004639   Thumb Code    52  memp.o(i.do_memp_free_pool)
    i.do_memp_malloc_pool                    0x0000468c   Section        0  memp.o(i.do_memp_malloc_pool)
    do_memp_malloc_pool                      0x0000468d   Thumb Code    62  memp.o(i.do_memp_malloc_pool)
    i.enet_get_rx_frame_size                 0x000046f0   Section        0  ethernetif.o(i.enet_get_rx_frame_size)
    enet_get_rx_frame_size                   0x000046f1   Thumb Code    16  ethernetif.o(i.enet_get_rx_frame_size)
    i.enet_get_tx_buffer                     0x00004700   Section        0  ethernetif.o(i.enet_get_tx_buffer)
    enet_get_tx_buffer                       0x00004701   Thumb Code     6  ethernetif.o(i.enet_get_tx_buffer)
    i.enet_init                              0x0000470c   Section        0  ethernetif.o(i.enet_init)
    enet_init                                0x0000470d   Thumb Code   200  ethernetif.o(i.enet_init)
    i.enet_read_frame                        0x000047d4   Section        0  ethernetif.o(i.enet_read_frame)
    enet_read_frame                          0x000047d5   Thumb Code    22  ethernetif.o(i.enet_read_frame)
    i.enet_send_frame                        0x000047ea   Section        0  ethernetif.o(i.enet_send_frame)
    enet_send_frame                          0x000047eb   Thumb Code    52  ethernetif.o(i.enet_send_frame)
    i.etharp_find_entry                      0x00004820   Section        0  etharp.o(i.etharp_find_entry)
    etharp_find_entry                        0x00004821   Thumb Code   450  etharp.o(i.etharp_find_entry)
    i.etharp_free_entry                      0x00004a80   Section        0  etharp.o(i.etharp_free_entry)
    etharp_free_entry                        0x00004a81   Thumb Code   112  etharp.o(i.etharp_free_entry)
    i.etharp_input                           0x00004af8   Section        0  etharp.o(i.etharp_input)
    i.etharp_output                          0x00004c1c   Section        0  etharp.o(i.etharp_output)
    i.etharp_output_to_arp_index             0x00004d98   Section        0  etharp.o(i.etharp_output_to_arp_index)
    etharp_output_to_arp_index               0x00004d99   Thumb Code   200  etharp.o(i.etharp_output_to_arp_index)
    i.etharp_query                           0x00004e94   Section        0  etharp.o(i.etharp_query)
    i.etharp_raw                             0x000050ac   Section        0  etharp.o(i.etharp_raw)
    etharp_raw                               0x000050ad   Thumb Code   194  etharp.o(i.etharp_raw)
    i.etharp_request                         0x000051b8   Section        0  etharp.o(i.etharp_request)
    i.etharp_request_dst                     0x000051d4   Section        0  etharp.o(i.etharp_request_dst)
    etharp_request_dst                       0x000051d5   Thumb Code    38  etharp.o(i.etharp_request_dst)
    i.etharp_tmr                             0x00005200   Section        0  etharp.o(i.etharp_tmr)
    i.etharp_update_arp_entry                0x000052e4   Section        0  etharp.o(i.etharp_update_arp_entry)
    etharp_update_arp_entry                  0x000052e5   Thumb Code   212  etharp.o(i.etharp_update_arp_entry)
    i.ethernet_input                         0x000053e0   Section        0  ethernet.o(i.ethernet_input)
    i.ethernet_output                        0x000054bc   Section        0  ethernet.o(i.ethernet_output)
    i.ethernetif_init                        0x0000555c   Section        0  ethernetif.o(i.ethernetif_init)
    i.ethernetif_input                       0x000055b8   Section        0  ethernetif.o(i.ethernetif_input)
    i.icmp_dest_unreach                      0x000055fc   Section        0  icmp.o(i.icmp_dest_unreach)
    i.icmp_input                             0x00005610   Section        0  icmp.o(i.icmp_input)
    i.icmp_send_response                     0x00005884   Section        0  icmp.o(i.icmp_send_response)
    icmp_send_response                       0x00005885   Thumb Code   142  icmp.o(i.icmp_send_response)
    i.icmp_time_exceeded                     0x00005940   Section        0  icmp.o(i.icmp_time_exceeded)
    i.inet_chksum                            0x00005952   Section        0  inet_chksum.o(i.inet_chksum)
    i.inet_chksum_pbuf                       0x00005966   Section        0  inet_chksum.o(i.inet_chksum_pbuf)
    i.inet_chksum_pseudo                     0x000059b8   Section        0  inet_chksum.o(i.inet_chksum_pseudo)
    i.inet_cksum_pseudo_base                 0x00005a04   Section        0  inet_chksum.o(i.inet_cksum_pseudo_base)
    inet_cksum_pseudo_base                   0x00005a05   Thumb Code   134  inet_chksum.o(i.inet_cksum_pseudo_base)
    i.ip4_addr_isbroadcast_u32               0x00005a8a   Section        0  ip4_addr.o(i.ip4_addr_isbroadcast_u32)
    i.ip4_frag                               0x00005ad8   Section        0  ip4_frag.o(i.ip4_frag)
    i.ip4_input                              0x00005d18   Section        0  ip4.o(i.ip4_input)
    i.ip4_output_if                          0x00005f60   Section        0  ip4.o(i.ip4_output_if)
    i.ip4_output_if_src                      0x00005f98   Section        0  ip4.o(i.ip4_output_if_src)
    i.ip4_reass                              0x00006100   Section        0  ip4_frag.o(i.ip4_reass)
    i.ip4_route                              0x000062c4   Section        0  ip4.o(i.ip4_route)
    i.ip_chksum_pseudo                       0x00006358   Section        0  inet_chksum.o(i.ip_chksum_pseudo)
    i.ip_frag_alloc_pbuf_custom_ref          0x0000637c   Section        0  ip4_frag.o(i.ip_frag_alloc_pbuf_custom_ref)
    ip_frag_alloc_pbuf_custom_ref            0x0000637d   Thumb Code    10  ip4_frag.o(i.ip_frag_alloc_pbuf_custom_ref)
    i.ip_frag_free_pbuf_custom_ref           0x00006388   Section        0  ip4_frag.o(i.ip_frag_free_pbuf_custom_ref)
    ip_frag_free_pbuf_custom_ref             0x00006389   Thumb Code    26  ip4_frag.o(i.ip_frag_free_pbuf_custom_ref)
    i.ip_reass_chain_frag_into_datagram_and_validate 0x000063b0   Section        0  ip4_frag.o(i.ip_reass_chain_frag_into_datagram_and_validate)
    ip_reass_chain_frag_into_datagram_and_validate 0x000063b1   Thumb Code   432  ip4_frag.o(i.ip_reass_chain_frag_into_datagram_and_validate)
    i.ip_reass_dequeue_datagram              0x00006620   Section        0  ip4_frag.o(i.ip_reass_dequeue_datagram)
    ip_reass_dequeue_datagram                0x00006621   Thumb Code    48  ip4_frag.o(i.ip_reass_dequeue_datagram)
    i.ip_reass_enqueue_new_datagram          0x00006670   Section        0  ip4_frag.o(i.ip_reass_enqueue_new_datagram)
    ip_reass_enqueue_new_datagram            0x00006671   Thumb Code    84  ip4_frag.o(i.ip_reass_enqueue_new_datagram)
    i.ip_reass_free_complete_datagram        0x000066c8   Section        0  ip4_frag.o(i.ip_reass_free_complete_datagram)
    ip_reass_free_complete_datagram          0x000066c9   Thumb Code   222  ip4_frag.o(i.ip_reass_free_complete_datagram)
    i.ip_reass_remove_oldest_datagram        0x00006808   Section        0  ip4_frag.o(i.ip_reass_remove_oldest_datagram)
    ip_reass_remove_oldest_datagram          0x00006809   Thumb Code   130  ip4_frag.o(i.ip_reass_remove_oldest_datagram)
    i.ip_reass_tmr                           0x00006890   Section        0  ip4_frag.o(i.ip_reass_tmr)
    i.ipfrag_free_pbuf_custom                0x000068cc   Section        0  ip4_frag.o(i.ipfrag_free_pbuf_custom)
    ipfrag_free_pbuf_custom                  0x000068cd   Thumb Code    50  ip4_frag.o(i.ipfrag_free_pbuf_custom)
    i.low_level_init                         0x00006918   Section        0  ethernetif.o(i.low_level_init)
    low_level_init                           0x00006919   Thumb Code    76  ethernetif.o(i.low_level_init)
    i.low_level_input                        0x00006964   Section        0  ethernetif.o(i.low_level_input)
    low_level_input                          0x00006965   Thumb Code   174  ethernetif.o(i.low_level_input)
    i.low_level_output                       0x00006a14   Section        0  ethernetif.o(i.low_level_output)
    low_level_output                         0x00006a15   Thumb Code   132  ethernetif.o(i.low_level_output)
    i.lwip_htonl                             0x00006ab4   Section        0  def.o(i.lwip_htonl)
    i.lwip_htons                             0x00006ace   Section        0  def.o(i.lwip_htons)
    i.lwip_init                              0x00006ada   Section        0  init.o(i.lwip_init)
    i.lwip_standard_chksum                   0x00006afa   Section        0  inet_chksum.o(i.lwip_standard_chksum)
    i.main                                   0x00006b58   Section        0  lwip_dhcp_bm.o(i.main)
    i.mem_free                               0x00006c58   Section        0  mem.o(i.mem_free)
    i.mem_init                               0x00006d38   Section        0  mem.o(i.mem_init)
    i.mem_malloc                             0x00006d94   Section        0  mem.o(i.mem_malloc)
    i.mem_trim                               0x00006f80   Section        0  mem.o(i.mem_trim)
    i.memp_free                              0x000070f0   Section        0  memp.o(i.memp_free)
    i.memp_init                              0x0000713c   Section        0  memp.o(i.memp_init)
    i.memp_init_pool                         0x0000715c   Section        0  memp.o(i.memp_init_pool)
    i.memp_malloc                            0x00007188   Section        0  memp.o(i.memp_malloc)
    i.netif_add                              0x000071d4   Section        0  netif.o(i.netif_add)
    i.netif_init                             0x00007288   Section        0  netif.o(i.netif_init)
    i.netif_issue_reports                    0x0000728a   Section        0  netif.o(i.netif_issue_reports)
    netif_issue_reports                      0x0000728b   Thumb Code    36  netif.o(i.netif_issue_reports)
    i.netif_set_addr                         0x000072ae   Section        0  netif.o(i.netif_set_addr)
    i.netif_set_default                      0x000072f8   Section        0  netif.o(i.netif_set_default)
    i.netif_set_gw                           0x00007308   Section        0  netif.o(i.netif_set_gw)
    i.netif_set_ipaddr                       0x00007318   Section        0  netif.o(i.netif_set_ipaddr)
    i.netif_set_netmask                      0x0000736c   Section        0  netif.o(i.netif_set_netmask)
    i.netif_set_up                           0x0000737c   Section        0  netif.o(i.netif_set_up)
    i.pbuf_alloc                             0x000073a8   Section        0  pbuf.o(i.pbuf_alloc)
    i.pbuf_alloced_custom                    0x0000770c   Section        0  pbuf.o(i.pbuf_alloced_custom)
    i.pbuf_cat                               0x000077bc   Section        0  pbuf.o(i.pbuf_cat)
    i.pbuf_chain                             0x0000788c   Section        0  pbuf.o(i.pbuf_chain)
    i.pbuf_clen                              0x000078a6   Section        0  pbuf.o(i.pbuf_clen)
    i.pbuf_copy                              0x000078b8   Section        0  pbuf.o(i.pbuf_copy)
    i.pbuf_copy_partial                      0x00007a50   Section        0  pbuf.o(i.pbuf_copy_partial)
    i.pbuf_free                              0x00007b34   Section        0  pbuf.o(i.pbuf_free)
    i.pbuf_header                            0x00007c74   Section        0  pbuf.o(i.pbuf_header)
    i.pbuf_header_force                      0x00007c86   Section        0  pbuf.o(i.pbuf_header_force)
    i.pbuf_header_impl                       0x00007c98   Section        0  pbuf.o(i.pbuf_header_impl)
    pbuf_header_impl                         0x00007c99   Thumb Code   184  pbuf.o(i.pbuf_header_impl)
    i.pbuf_realloc                           0x00007d8c   Section        0  pbuf.o(i.pbuf_realloc)
    i.pbuf_ref                               0x00007ecc   Section        0  pbuf.o(i.pbuf_ref)
    i.plug_holes                             0x00007eec   Section        0  mem.o(i.plug_holes)
    plug_holes                               0x00007eed   Thumb Code   178  mem.o(i.plug_holes)
    i.print_dhcp_state                       0x00008028   Section        0  lwip_dhcp_bm.o(i.print_dhcp_state)
    print_dhcp_state                         0x00008029   Thumb Code   228  lwip_dhcp_bm.o(i.print_dhcp_state)
    i.sys_arch_protect                       0x00008228   Section        0  sys_arch.o(i.sys_arch_protect)
    i.sys_arch_unprotect                     0x0000823a   Section        0  sys_arch.o(i.sys_arch_unprotect)
    i.sys_assert                             0x00008248   Section        0  sys_arch.o(i.sys_assert)
    i.sys_check_timeouts                     0x00008260   Section        0  timeouts.o(i.sys_check_timeouts)
    i.sys_now                                0x000082cc   Section        0  sys_arch.o(i.sys_now)
    i.sys_timeout                            0x000082d8   Section        0  timeouts.o(i.sys_timeout)
    i.sys_timeouts_init                      0x000083f8   Section        0  timeouts.o(i.sys_timeouts_init)
    i.tcp_abandon                            0x0000842c   Section        0  tcp.o(i.tcp_abandon)
    i.tcp_abort                              0x00008560   Section        0  tcp.o(i.tcp_abort)
    i.tcp_alloc                              0x00008570   Section        0  tcp.o(i.tcp_alloc)
    i.tcp_backlog_accepted                   0x00008644   Section        0  tcp.o(i.tcp_backlog_accepted)
    i.tcp_close                              0x000086a8   Section        0  tcp.o(i.tcp_close)
    i.tcp_close_shutdown                     0x000086c8   Section        0  tcp.o(i.tcp_close_shutdown)
    tcp_close_shutdown                       0x000086c9   Thumb Code   426  tcp.o(i.tcp_close_shutdown)
    i.tcp_create_segment                     0x000088a8   Section        0  tcp_out.o(i.tcp_create_segment)
    tcp_create_segment                       0x000088a9   Thumb Code   214  tcp_out.o(i.tcp_create_segment)
    i.tcp_eff_send_mss_impl                  0x00008998   Section        0  tcp.o(i.tcp_eff_send_mss_impl)
    i.tcp_enqueue_flags                      0x000089d4   Section        0  tcp_out.o(i.tcp_enqueue_flags)
    i.tcp_fasttmr                            0x00008be0   Section        0  tcp.o(i.tcp_fasttmr)
    i.tcp_getoptbyte                         0x00008c5c   Section        0  tcp_in.o(i.tcp_getoptbyte)
    tcp_getoptbyte                           0x00008c5d   Thumb Code    70  tcp_in.o(i.tcp_getoptbyte)
    i.tcp_init                               0x00008cb4   Section        0  tcp.o(i.tcp_init)
    i.tcp_input                              0x00008cb8   Section        0  tcp_in.o(i.tcp_input)
    i.tcp_keepalive                          0x000093d0   Section        0  tcp_out.o(i.tcp_keepalive)
    i.tcp_kill_prio                          0x0000945c   Section        0  tcp.o(i.tcp_kill_prio)
    tcp_kill_prio                            0x0000945d   Thumb Code    82  tcp.o(i.tcp_kill_prio)
    i.tcp_kill_state                         0x000094b8   Section        0  tcp.o(i.tcp_kill_state)
    tcp_kill_state                           0x000094b9   Thumb Code    86  tcp.o(i.tcp_kill_state)
    i.tcp_kill_timewait                      0x00009528   Section        0  tcp.o(i.tcp_kill_timewait)
    tcp_kill_timewait                        0x00009529   Thumb Code    54  tcp.o(i.tcp_kill_timewait)
    i.tcp_listen_closed                      0x00009568   Section        0  tcp.o(i.tcp_listen_closed)
    tcp_listen_closed                        0x00009569   Thumb Code    58  tcp.o(i.tcp_listen_closed)
    i.tcp_listen_input                       0x000095cc   Section        0  tcp_in.o(i.tcp_listen_input)
    tcp_listen_input                         0x000095cd   Thumb Code   326  tcp_in.o(i.tcp_listen_input)
    i.tcp_netif_ip_addr_changed              0x00009734   Section        0  tcp.o(i.tcp_netif_ip_addr_changed)
    i.tcp_netif_ip_addr_changed_pcblist      0x00009788   Section        0  tcp.o(i.tcp_netif_ip_addr_changed_pcblist)
    tcp_netif_ip_addr_changed_pcblist        0x00009789   Thumb Code    46  tcp.o(i.tcp_netif_ip_addr_changed_pcblist)
    i.tcp_next_iss                           0x000097b8   Section        0  tcp.o(i.tcp_next_iss)
    i.tcp_output                             0x000097d4   Section        0  tcp_out.o(i.tcp_output)
    i.tcp_output_alloc_header                0x00009a4c   Section        0  tcp_out.o(i.tcp_output_alloc_header)
    tcp_output_alloc_header                  0x00009a4d   Thumb Code   138  tcp_out.o(i.tcp_output_alloc_header)
    i.tcp_output_segment                     0x00009b08   Section        0  tcp_out.o(i.tcp_output_segment)
    tcp_output_segment                       0x00009b09   Thumb Code   222  tcp_out.o(i.tcp_output_segment)
    i.tcp_parseopt                           0x00009bec   Section        0  tcp_in.o(i.tcp_parseopt)
    tcp_parseopt                             0x00009bed   Thumb Code   174  tcp_in.o(i.tcp_parseopt)
    i.tcp_pcb_purge                          0x00009ca4   Section        0  tcp.o(i.tcp_pcb_purge)
    i.tcp_pcb_remove                         0x00009d04   Section        0  tcp.o(i.tcp_pcb_remove)
    i.tcp_process                            0x00009dc4   Section        0  tcp_in.o(i.tcp_process)
    tcp_process                              0x00009dc5   Thumb Code  1654  tcp_in.o(i.tcp_process)
    i.tcp_process_refused_data               0x0000a454   Section        0  tcp.o(i.tcp_process_refused_data)
    i.tcp_receive                            0x0000a4f0   Section        0  tcp_in.o(i.tcp_receive)
    tcp_receive                              0x0000a4f1   Thumb Code  1852  tcp_in.o(i.tcp_receive)
    i.tcp_recv_null                          0x0000acdc   Section        0  tcp.o(i.tcp_recv_null)
    i.tcp_recved                             0x0000ad0c   Section        0  tcp.o(i.tcp_recved)
    i.tcp_remove_listener                    0x0000add0   Section        0  tcp.o(i.tcp_remove_listener)
    tcp_remove_listener                      0x0000add1   Thumb Code    24  tcp.o(i.tcp_remove_listener)
    i.tcp_rexmit                             0x0000ade8   Section        0  tcp_out.o(i.tcp_rexmit)
    i.tcp_rexmit_fast                        0x0000ae42   Section        0  tcp_out.o(i.tcp_rexmit_fast)
    i.tcp_rexmit_rto                         0x0000aebe   Section        0  tcp_out.o(i.tcp_rexmit_rto)
    i.tcp_rst                                0x0000af04   Section        0  tcp_out.o(i.tcp_rst)
    i.tcp_seg_free                           0x0000afe0   Section        0  tcp.o(i.tcp_seg_free)
    i.tcp_segs_free                          0x0000affa   Section        0  tcp.o(i.tcp_segs_free)
    i.tcp_send_empty_ack                     0x0000b012   Section        0  tcp_out.o(i.tcp_send_empty_ack)
    i.tcp_send_fin                           0x0000b0a8   Section        0  tcp_out.o(i.tcp_send_fin)
    i.tcp_slowtmr                            0x0000b0f4   Section        0  tcp.o(i.tcp_slowtmr)
    i.tcp_timer_needed                       0x0000b638   Section        0  timeouts.o(i.tcp_timer_needed)
    i.tcp_timewait_input                     0x0000b670   Section        0  tcp_in.o(i.tcp_timewait_input)
    tcp_timewait_input                       0x0000b671   Thumb Code   134  tcp_in.o(i.tcp_timewait_input)
    i.tcp_tmr                                0x0000b714   Section        0  tcp.o(i.tcp_tmr)
    i.tcp_trigger_input_pcb_close            0x0000b738   Section        0  tcp_in.o(i.tcp_trigger_input_pcb_close)
    i.tcp_update_rcv_ann_wnd                 0x0000b74c   Section        0  tcp.o(i.tcp_update_rcv_ann_wnd)
    i.tcp_zero_window_probe                  0x0000b7c4   Section        0  tcp_out.o(i.tcp_zero_window_probe)
    i.tcpip_tcp_timer                        0x0000b8cc   Section        0  timeouts.o(i.tcpip_tcp_timer)
    tcpip_tcp_timer                          0x0000b8cd   Thumb Code    40  timeouts.o(i.tcpip_tcp_timer)
    i.time_init                              0x0000b904   Section        0  sys_arch.o(i.time_init)
    i.time_isr                               0x0000b978   Section        0  sys_arch.o(i.time_isr)
    i.udp_bind                               0x0000b988   Section        0  udp.o(i.udp_bind)
    i.udp_connect                            0x0000ba3c   Section        0  udp.o(i.udp_connect)
    i.udp_init                               0x0000bab8   Section        0  udp.o(i.udp_init)
    i.udp_input                              0x0000babc   Section        0  udp.o(i.udp_input)
    i.udp_input_local_match                  0x0000bc74   Section        0  udp.o(i.udp_input_local_match)
    udp_input_local_match                    0x0000bc75   Thumb Code    66  udp.o(i.udp_input_local_match)
    i.udp_netif_ip_addr_changed              0x0000bcbc   Section        0  udp.o(i.udp_netif_ip_addr_changed)
    i.udp_new                                0x0000bcec   Section        0  udp.o(i.udp_new)
    i.udp_new_port                           0x0000bd08   Section        0  udp.o(i.udp_new_port)
    udp_new_port                             0x0000bd09   Thumb Code    80  udp.o(i.udp_new_port)
    i.udp_recv                               0x0000bd60   Section        0  udp.o(i.udp_recv)
    i.udp_remove                             0x0000bd68   Section        0  udp.o(i.udp_remove)
    i.udp_sendto_if                          0x0000bdac   Section        0  udp.o(i.udp_sendto_if)
    i.udp_sendto_if_src                      0x0000be00   Section        0  udp.o(i.udp_sendto_if_src)
    .constdata                               0x0000bf48   Section        6  pin_mux.o(.constdata)
    .constdata                               0x0000bf50   Section       56  clock_config.o(.constdata)
    .constdata                               0x0000bf88   Section       56  fsl_uart.o(.constdata)
    s_uartBases                              0x0000bf88   Data          24  fsl_uart.o(.constdata)
    s_uartIRQ                                0x0000bfa0   Data           6  fsl_uart.o(.constdata)
    s_uartClock                              0x0000bfa8   Data          24  fsl_uart.o(.constdata)
    .constdata                               0x0000bfc0   Section       96  fsl_clock.o(.constdata)
    mcgModeMatrix                            0x0000bfc0   Data          64  fsl_clock.o(.constdata)
    fllFactorTable                           0x0000c000   Data          16  fsl_clock.o(.constdata)
    trimRange                                0x0000c010   Data          16  fsl_clock.o(.constdata)
    .constdata                               0x0000c020   Section       12  fsl_enet.o(.constdata)
    s_enetTxIrqId                            0x0000c024   Data           1  fsl_enet.o(.constdata)
    s_enetRxIrqId                            0x0000c025   Data           1  fsl_enet.o(.constdata)
    s_enetErrIrqId                           0x0000c026   Data           1  fsl_enet.o(.constdata)
    s_enetBases                              0x0000c028   Data           4  fsl_enet.o(.constdata)
    .constdata                               0x0000c02c   Section      180  memp.o(.constdata)
    .constdata                               0x0000c0e0   Section       80  tcp.o(.constdata)
    tcp_state_str                            0x0000c0e0   Data          44  tcp.o(.constdata)
    tcp_backoff                              0x0000c10c   Data          13  tcp.o(.constdata)
    tcp_persist_backoff                      0x0000c119   Data           7  tcp.o(.constdata)
    .constdata                               0x0000c130   Section       40  timeouts.o(.constdata)
    .constdata                               0x0000c158   Section        8  ip4_addr.o(.constdata)
    .constdata                               0x0000c160   Section       12  ethernet.o(.constdata)
    .conststring                             0x0000c16c   Section      277  fsl_enet.o(.conststring)
    .conststring                             0x0000c284   Section      104  memp.o(.conststring)
    .conststring                             0x0000c2ec   Section      109  tcp.o(.conststring)
    .conststring                             0x0000c35c   Section       85  tcp_out.o(.conststring)
    .conststring                             0x0000c3b4   Section      140  dhcp.o(.conststring)
    .conststring                             0x0000c440   Section       65  etharp.o(.conststring)
    .data                                    0x20000000   Section        4  system_mk64f12.o(.data)
    .data                                    0x20000004   Section        4  fsl_uart.o(.data)
    s_uartIsr                                0x20000004   Data           4  fsl_uart.o(.data)
    .data                                    0x20000008   Section       16  fsl_clock.o(.data)
    s_slowIrcFreq                            0x20000008   Data           4  fsl_clock.o(.data)
    s_fastIrcFreq                            0x2000000c   Data           4  fsl_clock.o(.data)
    .data                                    0x20000018   Section       20  fsl_enet.o(.data)
    s_ENETHandle                             0x20000018   Data           4  fsl_enet.o(.data)
    s_enetTxIsr                              0x2000001c   Data           4  fsl_enet.o(.data)
    s_enetRxIsr                              0x20000020   Data           4  fsl_enet.o(.data)
    s_enetErrIsr                             0x20000024   Data           4  fsl_enet.o(.data)
    s_enetTsIsr                              0x20000028   Data           4  fsl_enet.o(.data)
    .data                                    0x2000002c   Section        1  lwip_dhcp_bm.o(.data)
    dhcp_last_state                          0x2000002c   Data           1  lwip_dhcp_bm.o(.data)
    .data                                    0x20000030   Section       12  sys_arch.o(.data)
    _rand_value                              0x20000034   Data           4  sys_arch.o(.data)
    time_now                                 0x20000038   Data           4  sys_arch.o(.data)
    .data                                    0x2000003c   Section       12  mem.o(.data)
    ram                                      0x2000003c   Data           4  mem.o(.data)
    ram_end                                  0x20000040   Data           4  mem.o(.data)
    lfree                                    0x20000044   Data           4  mem.o(.data)
    .data                                    0x20000048   Section       36  memp.o(.data)
    memp_tab_UDP_PCB                         0x20000048   Data           4  memp.o(.data)
    memp_tab_TCP_PCB                         0x2000004c   Data           4  memp.o(.data)
    memp_tab_TCP_PCB_LISTEN                  0x20000050   Data           4  memp.o(.data)
    memp_tab_TCP_SEG                         0x20000054   Data           4  memp.o(.data)
    memp_tab_REASSDATA                       0x20000058   Data           4  memp.o(.data)
    memp_tab_FRAG_PBUF                       0x2000005c   Data           4  memp.o(.data)
    memp_tab_SYS_TIMEOUT                     0x20000060   Data           4  memp.o(.data)
    memp_tab_PBUF                            0x20000064   Data           4  memp.o(.data)
    memp_tab_PBUF_POOL                       0x20000068   Data           4  memp.o(.data)
    .data                                    0x2000006c   Section        9  netif.o(.data)
    netif_num                                0x20000074   Data           1  netif.o(.data)
    .data                                    0x20000078   Section       32  tcp.o(.data)
    tcp_port                                 0x20000078   Data           2  tcp.o(.data)
    tcp_timer                                0x20000091   Data           1  tcp.o(.data)
    tcp_timer_ctr                            0x20000092   Data           1  tcp.o(.data)
    iss                                      0x20000094   Data           4  tcp.o(.data)
    .data                                    0x20000098   Section       40  tcp_in.o(.data)
    tcphdr                                   0x20000098   Data           4  tcp_in.o(.data)
    tcphdr_optlen                            0x2000009c   Data           2  tcp_in.o(.data)
    tcphdr_opt1len                           0x2000009e   Data           2  tcp_in.o(.data)
    tcphdr_opt2                              0x200000a0   Data           4  tcp_in.o(.data)
    tcp_optidx                               0x200000a4   Data           2  tcp_in.o(.data)
    seqno                                    0x200000a8   Data           4  tcp_in.o(.data)
    ackno                                    0x200000ac   Data           4  tcp_in.o(.data)
    recv_acked                               0x200000b0   Data           2  tcp_in.o(.data)
    tcplen                                   0x200000b2   Data           2  tcp_in.o(.data)
    flags                                    0x200000b4   Data           1  tcp_in.o(.data)
    recv_flags                               0x200000b5   Data           1  tcp_in.o(.data)
    recv_data                                0x200000b8   Data           4  tcp_in.o(.data)
    .data                                    0x200000c0   Section       12  timeouts.o(.data)
    next_timeout                             0x200000c0   Data           4  timeouts.o(.data)
    timeouts_last_time                       0x200000c4   Data           4  timeouts.o(.data)
    tcpip_tcp_timer_active                   0x200000c8   Data           4  timeouts.o(.data)
    .data                                    0x200000cc   Section        8  udp.o(.data)
    udp_port                                 0x200000cc   Data           2  udp.o(.data)
    .data                                    0x200000d4   Section       16  dhcp.o(.data)
    dhcp_discover_request_options            0x200000d4   Data           4  dhcp.o(.data)
    dhcp_pcb                                 0x200000d8   Data           4  dhcp.o(.data)
    dhcp_pcb_refcount                        0x200000dc   Data           1  dhcp.o(.data)
    xid                                      0x200000e0   Data           4  dhcp.o(.data)
    .data                                    0x200000e4   Section        1  etharp.o(.data)
    etharp_cached_entry                      0x200000e4   Data           1  etharp.o(.data)
    .data                                    0x200000e6   Section        2  ip4.o(.data)
    ip_id                                    0x200000e6   Data           2  ip4.o(.data)
    .data                                    0x200000e8   Section        6  ip4_frag.o(.data)
    reassdatagrams                           0x200000e8   Data           4  ip4_frag.o(.data)
    ip_reass_pbufcount                       0x200000ec   Data           2  ip4_frag.o(.data)
    .bss                                     0x200000f0   Section       24  fsl_uart.o(.bss)
    s_uartHandle                             0x200000f0   Data          24  fsl_uart.o(.bss)
    .bss                                     0x20000108   Section       16  fsl_debug_console.o(.bss)
    s_debugConsole                           0x20000108   Data          16  fsl_debug_console.o(.bss)
    .bss                                     0x20000118   Section    13846  ethernetif.o(.bss)
    ethernetif_0                             0x20000118   Data       12328  ethernetif.o(.bss)
    ucBuffer                                 0x20003140   Data        1518  ethernetif.o(.bss)
    .bss                                     0x20003730   Section       24  ip.o(.bss)
    .bss                                     0x20003748   Section    22547  mem.o(.bss)
    .bss                                     0x20008f5b   Section    17039  memp.o(.bss)
    .bss                                     0x2000d1ec   Section       20  tcp_in.o(.bss)
    inseg                                    0x2000d1ec   Data          20  tcp_in.o(.bss)
    .bss                                     0x2000d200   Section       50  dhcp.o(.bss)
    .bss                                     0x2000d234   Section      240  etharp.o(.bss)
    arp_table                                0x2000d234   Data         240  etharp.o(.bss)

    Global Symbols

    Symbol Name                              Value     Ov Type        Size  Object(Section)

    BuildAttributes$$THM_ISAv4$E$P$D$K$B$S$7EM$VFPi3$EXTD16$VFPS$VFMA$PE$A:L22UL41UL21$X:L11$S22US41US21$IEEE1$IW$USESV6$~STKCKD$USESV7$~SHL$OSPACE$EBA8$MICROLIB$REQ8$PRES8$EABIv2 0x00000000   Number         0  anon$$obj.o ABSOLUTE
    Image$$VECTOR_ROM$$Base                  0x00000000   Number         0  anon$$obj.o ABSOLUTE
    __ARM_use_no_argv                        0x00000000   Number         0  lwip_dhcp_bm.o ABSOLUTE
    __Vectors                                0x00000000   Data           4  startup_mk64f12.o(RESET)
    __cpp_initialize__aeabi_                  - Undefined Weak Reference
    __cxa_finalize                            - Undefined Weak Reference
    __decompress                              - Undefined Weak Reference
    _clock_init                               - Undefined Weak Reference
    _microlib_exit                            - Undefined Weak Reference
    __Vectors_End                            0x00000400   Data           0  startup_mk64f12.o(RESET)
    __Vectors_Size                           0x00000400   Number         0  startup_mk64f12.o ABSOLUTE
    __main                                   0x00000411   Thumb Code     0  entry.o(.ARM.Collect$$$$00000000)
    _main_stk                                0x00000411   Thumb Code     0  entry4.o(.ARM.Collect$$$$00000003)
    _main_scatterload                        0x00000415   Thumb Code     0  entry5.o(.ARM.Collect$$$$00000004)
    __main_after_scatterload                 0x00000419   Thumb Code     0  entry5.o(.ARM.Collect$$$$00000004)
    _main_clock                              0x00000419   Thumb Code     0  entry7b.o(.ARM.Collect$$$$00000008)
    _main_cpp_init                           0x00000419   Thumb Code     0  entry8b.o(.ARM.Collect$$$$0000000A)
    _main_init                               0x00000419   Thumb Code     0  entry9a.o(.ARM.Collect$$$$0000000B)
    __rt_final_cpp                           0x00000421   Thumb Code     0  entry10a.o(.ARM.Collect$$$$0000000D)
    __rt_final_exit                          0x00000421   Thumb Code     0  entry11a.o(.ARM.Collect$$$$0000000F)
    Reset_Handler                            0x00000425   Thumb Code    24  startup_mk64f12.o(.text)
    NMI_Handler                              0x0000043d   Thumb Code     2  startup_mk64f12.o(.text)
    HardFault_Handler                        0x0000043f   Thumb Code     2  startup_mk64f12.o(.text)
    MemManage_Handler                        0x00000441   Thumb Code     2  startup_mk64f12.o(.text)
    BusFault_Handler                         0x00000443   Thumb Code     2  startup_mk64f12.o(.text)
    UsageFault_Handler                       0x00000445   Thumb Code     2  startup_mk64f12.o(.text)
    SVC_Handler                              0x00000447   Thumb Code     2  startup_mk64f12.o(.text)
    DebugMon_Handler                         0x00000449   Thumb Code     2  startup_mk64f12.o(.text)
    PendSV_Handler                           0x0000044b   Thumb Code     2  startup_mk64f12.o(.text)
    DMA0_IRQHandler                          0x0000044f   Thumb Code     4  startup_mk64f12.o(.text)
    DMA1_IRQHandler                          0x00000453   Thumb Code     4  startup_mk64f12.o(.text)
    DMA2_IRQHandler                          0x00000457   Thumb Code     4  startup_mk64f12.o(.text)
    DMA3_IRQHandler                          0x0000045b   Thumb Code     4  startup_mk64f12.o(.text)
    DMA4_IRQHandler                          0x0000045f   Thumb Code     4  startup_mk64f12.o(.text)
    DMA5_IRQHandler                          0x00000463   Thumb Code     4  startup_mk64f12.o(.text)
    DMA6_IRQHandler                          0x00000467   Thumb Code     4  startup_mk64f12.o(.text)
    DMA7_IRQHandler                          0x0000046b   Thumb Code     4  startup_mk64f12.o(.text)
    DMA8_IRQHandler                          0x0000046f   Thumb Code     4  startup_mk64f12.o(.text)
    DMA9_IRQHandler                          0x00000473   Thumb Code     4  startup_mk64f12.o(.text)
    DMA10_IRQHandler                         0x00000477   Thumb Code     4  startup_mk64f12.o(.text)
    DMA11_IRQHandler                         0x0000047b   Thumb Code     4  startup_mk64f12.o(.text)
    DMA12_IRQHandler                         0x0000047f   Thumb Code     4  startup_mk64f12.o(.text)
    DMA13_IRQHandler                         0x00000483   Thumb Code     4  startup_mk64f12.o(.text)
    DMA14_IRQHandler                         0x00000487   Thumb Code     4  startup_mk64f12.o(.text)
    DMA15_IRQHandler                         0x0000048b   Thumb Code     4  startup_mk64f12.o(.text)
    DMA_Error_IRQHandler                     0x0000048f   Thumb Code     4  startup_mk64f12.o(.text)
    I2C0_IRQHandler                          0x00000493   Thumb Code     4  startup_mk64f12.o(.text)
    I2C1_IRQHandler                          0x00000497   Thumb Code     4  startup_mk64f12.o(.text)
    SPI0_IRQHandler                          0x0000049b   Thumb Code     4  startup_mk64f12.o(.text)
    SPI1_IRQHandler                          0x0000049f   Thumb Code     4  startup_mk64f12.o(.text)
    I2S0_Tx_IRQHandler                       0x000004a3   Thumb Code     4  startup_mk64f12.o(.text)
    I2S0_Rx_IRQHandler                       0x000004a7   Thumb Code     4  startup_mk64f12.o(.text)
    UART0_LON_IRQHandler                     0x000004ab   Thumb Code     4  startup_mk64f12.o(.text)
    UART0_RX_TX_IRQHandler                   0x000004af   Thumb Code     4  startup_mk64f12.o(.text)
    UART0_ERR_IRQHandler                     0x000004b3   Thumb Code     4  startup_mk64f12.o(.text)
    UART1_RX_TX_IRQHandler                   0x000004b7   Thumb Code     4  startup_mk64f12.o(.text)
    UART1_ERR_IRQHandler                     0x000004bb   Thumb Code     4  startup_mk64f12.o(.text)
    UART2_RX_TX_IRQHandler                   0x000004bf   Thumb Code     4  startup_mk64f12.o(.text)
    UART2_ERR_IRQHandler                     0x000004c3   Thumb Code     4  startup_mk64f12.o(.text)
    UART3_RX_TX_IRQHandler                   0x000004c7   Thumb Code     4  startup_mk64f12.o(.text)
    UART3_ERR_IRQHandler                     0x000004cb   Thumb Code     4  startup_mk64f12.o(.text)
    SPI2_IRQHandler                          0x000004cf   Thumb Code     4  startup_mk64f12.o(.text)
    UART4_RX_TX_IRQHandler                   0x000004d3   Thumb Code     4  startup_mk64f12.o(.text)
    UART4_ERR_IRQHandler                     0x000004d7   Thumb Code     4  startup_mk64f12.o(.text)
    UART5_RX_TX_IRQHandler                   0x000004db   Thumb Code     4  startup_mk64f12.o(.text)
    UART5_ERR_IRQHandler                     0x000004df   Thumb Code     4  startup_mk64f12.o(.text)
    I2C2_IRQHandler                          0x000004e3   Thumb Code     4  startup_mk64f12.o(.text)
    CAN0_ORed_Message_buffer_IRQHandler      0x000004e7   Thumb Code     4  startup_mk64f12.o(.text)
    CAN0_Bus_Off_IRQHandler                  0x000004eb   Thumb Code     4  startup_mk64f12.o(.text)
    CAN0_Error_IRQHandler                    0x000004ef   Thumb Code     4  startup_mk64f12.o(.text)
    CAN0_Tx_Warning_IRQHandler               0x000004f3   Thumb Code     4  startup_mk64f12.o(.text)
    CAN0_Rx_Warning_IRQHandler               0x000004f7   Thumb Code     4  startup_mk64f12.o(.text)
    CAN0_Wake_Up_IRQHandler                  0x000004fb   Thumb Code     4  startup_mk64f12.o(.text)
    SDHC_IRQHandler                          0x000004ff   Thumb Code     4  startup_mk64f12.o(.text)
    ADC0_IRQHandler                          0x00000513   Thumb Code     0  startup_mk64f12.o(.text)
    ADC1_IRQHandler                          0x00000513   Thumb Code     0  startup_mk64f12.o(.text)
    CAN0_DriverIRQHandler                    0x00000513   Thumb Code     0  startup_mk64f12.o(.text)
    CMP0_IRQHandler                          0x00000513   Thumb Code     0  startup_mk64f12.o(.text)
    CMP1_IRQHandler                          0x00000513   Thumb Code     0  startup_mk64f12.o(.text)
    CMP2_IRQHandler                          0x00000513   Thumb Code     0  startup_mk64f12.o(.text)
    CMT_IRQHandler                           0x00000513   Thumb Code     0  startup_mk64f12.o(.text)
    DAC0_IRQHandler                          0x00000513   Thumb Code     0  startup_mk64f12.o(.text)
    DAC1_IRQHandler                          0x00000513   Thumb Code     0  startup_mk64f12.o(.text)
    DMA0_DriverIRQHandler                    0x00000513   Thumb Code     0  startup_mk64f12.o(.text)
    DMA10_DriverIRQHandler                   0x00000513   Thumb Code     0  startup_mk64f12.o(.text)
    DMA11_DriverIRQHandler                   0x00000513   Thumb Code     0  startup_mk64f12.o(.text)
    DMA12_DriverIRQHandler                   0x00000513   Thumb Code     0  startup_mk64f12.o(.text)
    DMA13_DriverIRQHandler                   0x00000513   Thumb Code     0  startup_mk64f12.o(.text)
    DMA14_DriverIRQHandler                   0x00000513   Thumb Code     0  startup_mk64f12.o(.text)
    DMA15_DriverIRQHandler                   0x00000513   Thumb Code     0  startup_mk64f12.o(.text)
    DMA1_DriverIRQHandler                    0x00000513   Thumb Code     0  startup_mk64f12.o(.text)
    DMA2_DriverIRQHandler                    0x00000513   Thumb Code     0  startup_mk64f12.o(.text)
    DMA3_DriverIRQHandler                    0x00000513   Thumb Code     0  startup_mk64f12.o(.text)
    DMA4_DriverIRQHandler                    0x00000513   Thumb Code     0  startup_mk64f12.o(.text)
    DMA5_DriverIRQHandler                    0x00000513   Thumb Code     0  startup_mk64f12.o(.text)
    DMA6_DriverIRQHandler                    0x00000513   Thumb Code     0  startup_mk64f12.o(.text)
    DMA7_DriverIRQHandler                    0x00000513   Thumb Code     0  startup_mk64f12.o(.text)
    DMA8_DriverIRQHandler                    0x00000513   Thumb Code     0  startup_mk64f12.o(.text)
    DMA9_DriverIRQHandler                    0x00000513   Thumb Code     0  startup_mk64f12.o(.text)
    DMA_Error_DriverIRQHandler               0x00000513   Thumb Code     0  startup_mk64f12.o(.text)
    DefaultISR                               0x00000513   Thumb Code     0  startup_mk64f12.o(.text)
    ENET_1588_Timer_DriverIRQHandler         0x00000513   Thumb Code     0  startup_mk64f12.o(.text)
    ENET_Error_DriverIRQHandler              0x00000513   Thumb Code     0  startup_mk64f12.o(.text)
    ENET_Receive_DriverIRQHandler            0x00000513   Thumb Code     0  startup_mk64f12.o(.text)
    ENET_Transmit_DriverIRQHandler           0x00000513   Thumb Code     0  startup_mk64f12.o(.text)
    FTFE_IRQHandler                          0x00000513   Thumb Code     0  startup_mk64f12.o(.text)
    FTM0_IRQHandler                          0x00000513   Thumb Code     0  startup_mk64f12.o(.text)
    FTM1_IRQHandler                          0x00000513   Thumb Code     0  startup_mk64f12.o(.text)
    FTM2_IRQHandler                          0x00000513   Thumb Code     0  startup_mk64f12.o(.text)
    FTM3_IRQHandler                          0x00000513   Thumb Code     0  startup_mk64f12.o(.text)
    I2C0_DriverIRQHandler                    0x00000513   Thumb Code     0  startup_mk64f12.o(.text)
    I2C1_DriverIRQHandler                    0x00000513   Thumb Code     0  startup_mk64f12.o(.text)
    I2C2_DriverIRQHandler                    0x00000513   Thumb Code     0  startup_mk64f12.o(.text)
    I2S0_Rx_DriverIRQHandler                 0x00000513   Thumb Code     0  startup_mk64f12.o(.text)
    I2S0_Tx_DriverIRQHandler                 0x00000513   Thumb Code     0  startup_mk64f12.o(.text)
    LLWU_IRQHandler                          0x00000513   Thumb Code     0  startup_mk64f12.o(.text)
    LPTMR0_IRQHandler                        0x00000513   Thumb Code     0  startup_mk64f12.o(.text)
    LVD_LVW_IRQHandler                       0x00000513   Thumb Code     0  startup_mk64f12.o(.text)
    MCG_IRQHandler                           0x00000513   Thumb Code     0  startup_mk64f12.o(.text)
    MCM_IRQHandler                           0x00000513   Thumb Code     0  startup_mk64f12.o(.text)
    PDB0_IRQHandler                          0x00000513   Thumb Code     0  startup_mk64f12.o(.text)
    PIT0_IRQHandler                          0x00000513   Thumb Code     0  startup_mk64f12.o(.text)
    PIT1_IRQHandler                          0x00000513   Thumb Code     0  startup_mk64f12.o(.text)
    PIT2_IRQHandler                          0x00000513   Thumb Code     0  startup_mk64f12.o(.text)
    PIT3_IRQHandler                          0x00000513   Thumb Code     0  startup_mk64f12.o(.text)
    PORTA_IRQHandler                         0x00000513   Thumb Code     0  startup_mk64f12.o(.text)
    PORTB_IRQHandler                         0x00000513   Thumb Code     0  startup_mk64f12.o(.text)
    PORTC_IRQHandler                         0x00000513   Thumb Code     0  startup_mk64f12.o(.text)
    PORTD_IRQHandler                         0x00000513   Thumb Code     0  startup_mk64f12.o(.text)
    PORTE_IRQHandler                         0x00000513   Thumb Code     0  startup_mk64f12.o(.text)
    RNG_IRQHandler                           0x00000513   Thumb Code     0  startup_mk64f12.o(.text)
    RTC_IRQHandler                           0x00000513   Thumb Code     0  startup_mk64f12.o(.text)
    RTC_Seconds_IRQHandler                   0x00000513   Thumb Code     0  startup_mk64f12.o(.text)
    Read_Collision_IRQHandler                0x00000513   Thumb Code     0  startup_mk64f12.o(.text)
    Reserved71_IRQHandler                    0x00000513   Thumb Code     0  startup_mk64f12.o(.text)
    SDHC_DriverIRQHandler                    0x00000513   Thumb Code     0  startup_mk64f12.o(.text)
    SPI0_DriverIRQHandler                    0x00000513   Thumb Code     0  startup_mk64f12.o(.text)
    SPI1_DriverIRQHandler                    0x00000513   Thumb Code     0  startup_mk64f12.o(.text)
    SPI2_DriverIRQHandler                    0x00000513   Thumb Code     0  startup_mk64f12.o(.text)
    SWI_IRQHandler                           0x00000513   Thumb Code     0  startup_mk64f12.o(.text)
    UART0_ERR_DriverIRQHandler               0x00000513   Thumb Code     0  startup_mk64f12.o(.text)
    UART0_LON_DriverIRQHandler               0x00000513   Thumb Code     0  startup_mk64f12.o(.text)
    UART1_ERR_DriverIRQHandler               0x00000513   Thumb Code     0  startup_mk64f12.o(.text)
    UART2_ERR_DriverIRQHandler               0x00000513   Thumb Code     0  startup_mk64f12.o(.text)
    UART3_ERR_DriverIRQHandler               0x00000513   Thumb Code     0  startup_mk64f12.o(.text)
    UART4_ERR_DriverIRQHandler               0x00000513   Thumb Code     0  startup_mk64f12.o(.text)
    UART5_ERR_DriverIRQHandler               0x00000513   Thumb Code     0  startup_mk64f12.o(.text)
    USB0_IRQHandler                          0x00000513   Thumb Code     0  startup_mk64f12.o(.text)
    USBDCD_IRQHandler                        0x00000513   Thumb Code     0  startup_mk64f12.o(.text)
    WDOG_EWM_IRQHandler                      0x00000513   Thumb Code     0  startup_mk64f12.o(.text)
    __aeabi_uldivmod                         0x000005e9   Thumb Code    98  uldiv.o(.text)
    __aeabi_memcpy                           0x0000064b   Thumb Code    36  memcpya.o(.text)
    __aeabi_memcpy4                          0x0000064b   Thumb Code     0  memcpya.o(.text)
    __aeabi_memcpy8                          0x0000064b   Thumb Code     0  memcpya.o(.text)
    __aeabi_memset                           0x0000066f   Thumb Code    14  memseta.o(.text)
    __aeabi_memset4                          0x0000066f   Thumb Code     0  memseta.o(.text)
    __aeabi_memset8                          0x0000066f   Thumb Code     0  memseta.o(.text)
    __aeabi_memclr                           0x0000067d   Thumb Code     4  memseta.o(.text)
    __aeabi_memclr4                          0x0000067d   Thumb Code     0  memseta.o(.text)
    __aeabi_memclr8                          0x0000067d   Thumb Code     0  memseta.o(.text)
    _memset$wrapper                          0x00000681   Thumb Code    18  memseta.o(.text)
    strlen                                   0x00000693   Thumb Code    14  strlen.o(.text)
    memcmp                                   0x000006a1   Thumb Code    26  memcmp.o(.text)
    __aeabi_llsl                             0x000006bb   Thumb Code    30  llshl.o(.text)
    _ll_shift_l                              0x000006bb   Thumb Code     0  llshl.o(.text)
    __aeabi_llsr                             0x000006d9   Thumb Code    32  llushr.o(.text)
    _ll_ushift_r                             0x000006d9   Thumb Code     0  llushr.o(.text)
    __scatterload                            0x000006f9   Thumb Code    28  init.o(.text)
    __scatterload_rt2                        0x000006f9   Thumb Code     0  init.o(.text)
    BOARD_BootClockRUN                       0x0000071d   Thumb Code    78  clock_config.o(i.BOARD_BootClockRUN)
    BOARD_InitDebugConsole                   0x00000789   Thumb Code    24  board.o(i.BOARD_InitDebugConsole)
    BOARD_InitPins                           0x000007a5   Thumb Code   212  pin_mux.o(i.BOARD_InitPins)
    CLOCK_BootToPeeMode                      0x00000891   Thumb Code    68  fsl_clock.o(i.CLOCK_BootToPeeMode)
    CLOCK_EnablePll0                         0x00000949   Thumb Code    78  fsl_clock.o(i.CLOCK_EnablePll0)
    CLOCK_GetCoreSysClkFreq                  0x000009e1   Thumb Code    22  fsl_clock.o(i.CLOCK_GetCoreSysClkFreq)
    CLOCK_GetEr32kClkFreq                    0x000009fd   Thumb Code    86  fsl_clock.o(i.CLOCK_GetEr32kClkFreq)
    CLOCK_GetFixedFreqClkFreq                0x00000aa9   Thumb Code    28  fsl_clock.o(i.CLOCK_GetFixedFreqClkFreq)
    CLOCK_GetFllFreq                         0x00000b35   Thumb Code    66  fsl_clock.o(i.CLOCK_GetFllFreq)
    CLOCK_GetFreq                            0x00000ba1   Thumb Code   190  fsl_clock.o(i.CLOCK_GetFreq)
    CLOCK_GetInternalRefClkFreq              0x00000c69   Thumb Code    22  fsl_clock.o(i.CLOCK_GetInternalRefClkFreq)
    CLOCK_GetOsc0ErClkFreq                   0x00000d6d   Thumb Code    42  fsl_clock.o(i.CLOCK_GetOsc0ErClkFreq)
    CLOCK_GetOutClkFreq                      0x00000e09   Thumb Code    56  fsl_clock.o(i.CLOCK_GetOutClkFreq)
    CLOCK_GetPll0Freq                        0x00000e45   Thumb Code    68  fsl_clock.o(i.CLOCK_GetPll0Freq)
    CLOCK_GetPllFllSelClkFreq                0x00000edd   Thumb Code    46  fsl_clock.o(i.CLOCK_GetPllFllSelClkFreq)
    CLOCK_InitOsc0                           0x00000f15   Thumb Code    98  fsl_clock.o(i.CLOCK_InitOsc0)
    CLOCK_SetExternalRefClkConfig            0x00000f81   Thumb Code    56  fsl_clock.o(i.CLOCK_SetExternalRefClkConfig)
    CLOCK_SetInternalRefClkConfig            0x00000fbd   Thumb Code   148  fsl_clock.o(i.CLOCK_SetInternalRefClkConfig)
    CLOCK_SetPbeMode                         0x00001055   Thumb Code   124  fsl_clock.o(i.CLOCK_SetPbeMode)
    CLOCK_SetSimConfig                       0x00001119   Thumb Code    38  fsl_clock.o(i.CLOCK_SetSimConfig)
    DbgConsole_Init                          0x000011f1   Thumb Code   140  fsl_debug_console.o(i.DbgConsole_Init)
    DbgConsole_Printf                        0x00001289   Thumb Code    44  fsl_debug_console.o(i.DbgConsole_Printf)
    DbgConsole_Putchar                       0x00001521   Thumb Code    30  fsl_debug_console.o(i.DbgConsole_Putchar)
    ENET_1588_Timer_IRQHandler               0x00001545   Thumb Code    16  fsl_enet.o(i.ENET_1588_Timer_IRQHandler)
    ENET_ErrorIRQHandler                     0x00001565   Thumb Code   108  fsl_enet.o(i.ENET_ErrorIRQHandler)
    ENET_Error_IRQHandler                    0x00001615   Thumb Code    16  fsl_enet.o(i.ENET_Error_IRQHandler)
    ENET_GetDefaultConfig                    0x00001631   Thumb Code    44  fsl_enet.o(i.ENET_GetDefaultConfig)
    ENET_GetInstance                         0x0000169d   Thumb Code    48  fsl_enet.o(i.ENET_GetInstance)
    ENET_GetRxFrameSize                      0x0000172d   Thumb Code   144  fsl_enet.o(i.ENET_GetRxFrameSize)
    ENET_Init                                0x00001819   Thumb Code   386  fsl_enet.o(i.ENET_Init)
    ENET_ReadFrame                           0x00001ac9   Thumb Code   208  fsl_enet.o(i.ENET_ReadFrame)
    ENET_ReceiveIRQHandler                   0x00001bed   Thumb Code    58  fsl_enet.o(i.ENET_ReceiveIRQHandler)
    ENET_Receive_IRQHandler                  0x00001c69   Thumb Code    16  fsl_enet.o(i.ENET_Receive_IRQHandler)
    ENET_SendFrame                           0x00001c85   Thumb Code   298  fsl_enet.o(i.ENET_SendFrame)
    ENET_SetMacAddr                          0x00001edd   Thumb Code    44  fsl_enet.o(i.ENET_SetMacAddr)
    ENET_SetSMI                              0x00002179   Thumb Code    92  fsl_enet.o(i.ENET_SetSMI)
    ENET_StartSMIRead                        0x000022dd   Thumb Code    44  fsl_enet.o(i.ENET_StartSMIRead)
    ENET_StartSMIWrite                       0x00002309   Thumb Code    52  fsl_enet.o(i.ENET_StartSMIWrite)
    ENET_TransmitIRQHandler                  0x0000233d   Thumb Code    58  fsl_enet.o(i.ENET_TransmitIRQHandler)
    ENET_Transmit_IRQHandler                 0x000023b9   Thumb Code    16  fsl_enet.o(i.ENET_Transmit_IRQHandler)
    PHY_GetLinkSpeedDuplex                   0x00002485   Thumb Code   100  fsl_phy.o(i.PHY_GetLinkSpeedDuplex)
    PHY_GetLinkStatus                        0x00002501   Thumb Code    62  fsl_phy.o(i.PHY_GetLinkStatus)
    PHY_Init                                 0x00002559   Thumb Code   200  fsl_phy.o(i.PHY_Init)
    PHY_Read                                 0x0000262d   Thumb Code   104  fsl_phy.o(i.PHY_Read)
    PHY_Write                                0x000026b1   Thumb Code    84  fsl_phy.o(i.PHY_Write)
    SysTick_Handler                          0x0000277f   Thumb Code     8  lwip_dhcp_bm.o(i.SysTick_Handler)
    SystemInit                               0x00002789   Thumb Code    34  system_mk64f12.o(i.SystemInit)
    UART0_DriverIRQHandler                   0x000027b5   Thumb Code    16  fsl_uart.o(i.UART0_DriverIRQHandler)
    UART0_RX_TX_DriverIRQHandler             0x000027d1   Thumb Code     8  fsl_uart.o(i.UART0_RX_TX_DriverIRQHandler)
    UART1_DriverIRQHandler                   0x000027d9   Thumb Code    16  fsl_uart.o(i.UART1_DriverIRQHandler)
    UART1_RX_TX_DriverIRQHandler             0x000027f5   Thumb Code     8  fsl_uart.o(i.UART1_RX_TX_DriverIRQHandler)
    UART2_DriverIRQHandler                   0x000027fd   Thumb Code    16  fsl_uart.o(i.UART2_DriverIRQHandler)
    UART2_RX_TX_DriverIRQHandler             0x00002819   Thumb Code     8  fsl_uart.o(i.UART2_RX_TX_DriverIRQHandler)
    UART3_DriverIRQHandler                   0x00002821   Thumb Code    16  fsl_uart.o(i.UART3_DriverIRQHandler)
    UART3_RX_TX_DriverIRQHandler             0x0000283d   Thumb Code     8  fsl_uart.o(i.UART3_RX_TX_DriverIRQHandler)
    UART4_DriverIRQHandler                   0x00002845   Thumb Code    16  fsl_uart.o(i.UART4_DriverIRQHandler)
    UART4_RX_TX_DriverIRQHandler             0x00002861   Thumb Code     8  fsl_uart.o(i.UART4_RX_TX_DriverIRQHandler)
    UART5_DriverIRQHandler                   0x00002869   Thumb Code    16  fsl_uart.o(i.UART5_DriverIRQHandler)
    UART5_RX_TX_DriverIRQHandler             0x00002885   Thumb Code     8  fsl_uart.o(i.UART5_RX_TX_DriverIRQHandler)
    UART_GetDefaultConfig                    0x0000288d   Thumb Code    46  fsl_uart.o(i.UART_GetDefaultConfig)
    UART_GetInstance                         0x000028fd   Thumb Code    50  fsl_uart.o(i.UART_GetInstance)
    UART_GetStatusFlags                      0x00002989   Thumb Code    24  fsl_uart.o(i.UART_GetStatusFlags)
    UART_Init                                0x000029a1   Thumb Code   430  fsl_uart.o(i.UART_Init)
    UART_ReadBlocking                        0x00002c45   Thumb Code   112  fsl_uart.o(i.UART_ReadBlocking)
    UART_WriteBlocking                       0x00002cf5   Thumb Code    32  fsl_uart.o(i.UART_WriteBlocking)
    __aeabi_assert                           0x00002d15   Thumb Code    24  fsl_common.o(i.__aeabi_assert)
    __scatterload_copy                       0x00002d59   Thumb Code    14  handlers.o(i.__scatterload_copy)
    __scatterload_null                       0x00002d67   Thumb Code     2  handlers.o(i.__scatterload_null)
    __scatterload_zeroinit                   0x00002d69   Thumb Code    14  handlers.o(i.__scatterload_zeroinit)
    dhcp_arp_reply                           0x00002d95   Thumb Code    60  dhcp.o(i.dhcp_arp_reply)
    dhcp_coarse_tmr                          0x00002f91   Thumb Code   116  dhcp.o(i.dhcp_coarse_tmr)
    dhcp_fine_tmr                            0x00003515   Thumb Code    58  dhcp.o(i.dhcp_fine_tmr)
    dhcp_release                             0x000040b1   Thumb Code   174  dhcp.o(i.dhcp_release)
    dhcp_renew                               0x00004169   Thumb Code   198  dhcp.o(i.dhcp_renew)
    dhcp_start                               0x0000435d   Thumb Code   198  dhcp.o(i.dhcp_start)
    dhcp_stop                                0x00004485   Thumb Code    64  dhcp.o(i.dhcp_stop)
    dhcp_supplied_address                    0x000044f5   Thumb Code    34  dhcp.o(i.dhcp_supplied_address)
    etharp_input                             0x00004af9   Thumb Code   272  etharp.o(i.etharp_input)
    etharp_output                            0x00004c1d   Thumb Code   324  etharp.o(i.etharp_output)
    etharp_query                             0x00004e95   Thumb Code   448  etharp.o(i.etharp_query)
    etharp_request                           0x000051b9   Thumb Code    22  etharp.o(i.etharp_request)
    etharp_tmr                               0x00005201   Thumb Code   224  etharp.o(i.etharp_tmr)
    ethernet_input                           0x000053e1   Thumb Code   216  ethernet.o(i.ethernet_input)
    ethernet_output                          0x000054bd   Thumb Code   108  ethernet.o(i.ethernet_output)
    ethernetif_init                          0x0000555d   Thumb Code    60  ethernetif.o(i.ethernetif_init)
    ethernetif_input                         0x000055b9   Thumb Code    52  ethernetif.o(i.ethernetif_input)
    icmp_dest_unreach                        0x000055fd   Thumb Code    18  icmp.o(i.icmp_dest_unreach)
    icmp_input                               0x00005611   Thumb Code   516  icmp.o(i.icmp_input)
    icmp_time_exceeded                       0x00005941   Thumb Code    18  icmp.o(i.icmp_time_exceeded)
    inet_chksum                              0x00005953   Thumb Code    20  inet_chksum.o(i.inet_chksum)
    inet_chksum_pbuf                         0x00005967   Thumb Code    82  inet_chksum.o(i.inet_chksum_pbuf)
    inet_chksum_pseudo                       0x000059b9   Thumb Code    76  inet_chksum.o(i.inet_chksum_pseudo)
    ip4_addr_isbroadcast_u32                 0x00005a8b   Thumb Code    78  ip4_addr.o(i.ip4_addr_isbroadcast_u32)
    ip4_frag                                 0x00005ad9   Thumb Code   470  ip4_frag.o(i.ip4_frag)
    ip4_input                                0x00005d19   Thumb Code   574  ip4.o(i.ip4_input)
    ip4_output_if                            0x00005f61   Thumb Code    54  ip4.o(i.ip4_output_if)
    ip4_output_if_src                        0x00005f99   Thumb Code   290  ip4.o(i.ip4_output_if_src)
    ip4_reass                                0x00006101   Thumb Code   442  ip4_frag.o(i.ip4_reass)
    ip4_route                                0x000062c5   Thumb Code   138  ip4.o(i.ip4_route)
    ip_chksum_pseudo                         0x00006359   Thumb Code    36  inet_chksum.o(i.ip_chksum_pseudo)
    ip_reass_tmr                             0x00006891   Thumb Code    56  ip4_frag.o(i.ip_reass_tmr)
    lwip_htonl                               0x00006ab5   Thumb Code    26  def.o(i.lwip_htonl)
    lwip_htons                               0x00006acf   Thumb Code    12  def.o(i.lwip_htons)
    lwip_init                                0x00006adb   Thumb Code    32  init.o(i.lwip_init)
    lwip_standard_chksum                     0x00006afb   Thumb Code    94  inet_chksum.o(i.lwip_standard_chksum)
    main                                     0x00006b59   Thumb Code   120  lwip_dhcp_bm.o(i.main)
    mem_free                                 0x00006c59   Thumb Code   132  mem.o(i.mem_free)
    mem_init                                 0x00006d39   Thumb Code    74  mem.o(i.mem_init)
    mem_malloc                               0x00006d95   Thumb Code   320  mem.o(i.mem_malloc)
    mem_trim                                 0x00006f81   Thumb Code   300  mem.o(i.mem_trim)
    memp_free                                0x000070f1   Thumb Code    42  memp.o(i.memp_free)
    memp_init                                0x0000713d   Thumb Code    26  memp.o(i.memp_init)
    memp_init_pool                           0x0000715d   Thumb Code    44  memp.o(i.memp_init_pool)
    memp_malloc                              0x00007189   Thumb Code    38  memp.o(i.memp_malloc)
    netif_add                                0x000071d5   Thumb Code   148  netif.o(i.netif_add)
    netif_init                               0x00007289   Thumb Code     2  netif.o(i.netif_init)
    netif_set_addr                           0x000072af   Thumb Code    72  netif.o(i.netif_set_addr)
    netif_set_default                        0x000072f9   Thumb Code    10  netif.o(i.netif_set_default)
    netif_set_gw                             0x00007309   Thumb Code    16  netif.o(i.netif_set_gw)
    netif_set_ipaddr                         0x00007319   Thumb Code    80  netif.o(i.netif_set_ipaddr)
    netif_set_netmask                        0x0000736d   Thumb Code    16  netif.o(i.netif_set_netmask)
    netif_set_up                             0x0000737d   Thumb Code    44  netif.o(i.netif_set_up)
    pbuf_alloc                               0x000073a9   Thumb Code   548  pbuf.o(i.pbuf_alloc)
    pbuf_alloced_custom                      0x0000770d   Thumb Code   138  pbuf.o(i.pbuf_alloced_custom)
    pbuf_cat                                 0x000077bd   Thumb Code    88  pbuf.o(i.pbuf_cat)
    pbuf_chain                               0x0000788d   Thumb Code    26  pbuf.o(i.pbuf_chain)
    pbuf_clen                                0x000078a7   Thumb Code    18  pbuf.o(i.pbuf_clen)
    pbuf_copy                                0x000078b9   Thumb Code   248  pbuf.o(i.pbuf_copy)
    pbuf_copy_partial                        0x00007a51   Thumb Code   158  pbuf.o(i.pbuf_copy_partial)
    pbuf_free                                0x00007b35   Thumb Code   222  pbuf.o(i.pbuf_free)
    pbuf_header                              0x00007c75   Thumb Code    18  pbuf.o(i.pbuf_header)
    pbuf_header_force                        0x00007c87   Thumb Code    18  pbuf.o(i.pbuf_header_force)
    pbuf_realloc                             0x00007d8d   Thumb Code   194  pbuf.o(i.pbuf_realloc)
    pbuf_ref                                 0x00007ecd   Thumb Code    30  pbuf.o(i.pbuf_ref)
    sys_arch_protect                         0x00008229   Thumb Code    18  sys_arch.o(i.sys_arch_protect)
    sys_arch_unprotect                       0x0000823b   Thumb Code    14  sys_arch.o(i.sys_arch_unprotect)
    sys_assert                               0x00008249   Thumb Code    18  sys_arch.o(i.sys_assert)
    sys_check_timeouts                       0x00008261   Thumb Code    98  timeouts.o(i.sys_check_timeouts)
    sys_now                                  0x000082cd   Thumb Code     6  sys_arch.o(i.sys_now)
    sys_timeout                              0x000082d9   Thumb Code   214  timeouts.o(i.sys_timeout)
    sys_timeouts_init                        0x000083f9   Thumb Code    38  timeouts.o(i.sys_timeouts_init)
    tcp_abandon                              0x0000842d   Thumb Code   238  tcp.o(i.tcp_abandon)
    tcp_abort                                0x00008561   Thumb Code    14  tcp.o(i.tcp_abort)
    tcp_alloc                                0x00008571   Thumb Code   194  tcp.o(i.tcp_alloc)
    tcp_backlog_accepted                     0x00008645   Thumb Code    64  tcp.o(i.tcp_backlog_accepted)
    tcp_close                                0x000086a9   Thumb Code    32  tcp.o(i.tcp_close)
    tcp_eff_send_mss_impl                    0x00008999   Thumb Code    58  tcp.o(i.tcp_eff_send_mss_impl)
    tcp_enqueue_flags                        0x000089d5   Thumb Code   352  tcp_out.o(i.tcp_enqueue_flags)
    tcp_fasttmr                              0x00008be1   Thumb Code   112  tcp.o(i.tcp_fasttmr)
    tcp_init                                 0x00008cb5   Thumb Code     2  tcp.o(i.tcp_init)
    tcp_input                                0x00008cb9   Thumb Code  1746  tcp_in.o(i.tcp_input)
    tcp_keepalive                            0x000093d1   Thumb Code   138  tcp_out.o(i.tcp_keepalive)
    tcp_netif_ip_addr_changed                0x00009735   Thumb Code    70  tcp.o(i.tcp_netif_ip_addr_changed)
    tcp_next_iss                             0x000097b9   Thumb Code    20  tcp.o(i.tcp_next_iss)
    tcp_output                               0x000097d5   Thumb Code   562  tcp_out.o(i.tcp_output)
    tcp_pcb_purge                            0x00009ca5   Thumb Code    94  tcp.o(i.tcp_pcb_purge)
    tcp_pcb_remove                           0x00009d05   Thumb Code   140  tcp.o(i.tcp_pcb_remove)
    tcp_process_refused_data                 0x0000a455   Thumb Code   154  tcp.o(i.tcp_process_refused_data)
    tcp_recv_null                            0x0000acdd   Thumb Code    46  tcp.o(i.tcp_recv_null)
    tcp_recved                               0x0000ad0d   Thumb Code   118  tcp.o(i.tcp_recved)
    tcp_rexmit                               0x0000ade9   Thumb Code    90  tcp_out.o(i.tcp_rexmit)
    tcp_rexmit_fast                          0x0000ae43   Thumb Code   124  tcp_out.o(i.tcp_rexmit_fast)
    tcp_rexmit_rto                           0x0000aebf   Thumb Code    68  tcp_out.o(i.tcp_rexmit_rto)
    tcp_rst                                  0x0000af05   Thumb Code   172  tcp_out.o(i.tcp_rst)
    tcp_seg_free                             0x0000afe1   Thumb Code    26  tcp.o(i.tcp_seg_free)
    tcp_segs_free                            0x0000affb   Thumb Code    24  tcp.o(i.tcp_segs_free)
    tcp_send_empty_ack                       0x0000b013   Thumb Code   150  tcp_out.o(i.tcp_send_empty_ack)
    tcp_send_fin                             0x0000b0a9   Thumb Code    74  tcp_out.o(i.tcp_send_fin)
    tcp_slowtmr                              0x0000b0f5   Thumb Code   964  tcp.o(i.tcp_slowtmr)
    tcp_timer_needed                         0x0000b639   Thumb Code    38  timeouts.o(i.tcp_timer_needed)
    tcp_tmr                                  0x0000b715   Thumb Code    30  tcp.o(i.tcp_tmr)
    tcp_trigger_input_pcb_close              0x0000b739   Thumb Code    14  tcp_in.o(i.tcp_trigger_input_pcb_close)
    tcp_update_rcv_ann_wnd                   0x0000b74d   Thumb Code    90  tcp.o(i.tcp_update_rcv_ann_wnd)
    tcp_zero_window_probe                    0x0000b7c5   Thumb Code   262  tcp_out.o(i.tcp_zero_window_probe)
    time_init                                0x0000b905   Thumb Code   102  sys_arch.o(i.time_init)
    time_isr                                 0x0000b979   Thumb Code    12  sys_arch.o(i.time_isr)
    udp_bind                                 0x0000b989   Thumb Code   172  udp.o(i.udp_bind)
    udp_connect                              0x0000ba3d   Thumb Code   118  udp.o(i.udp_connect)
    udp_init                                 0x0000bab9   Thumb Code     2  udp.o(i.udp_init)
    udp_input                                0x0000babd   Thumb Code   410  udp.o(i.udp_input)
    udp_netif_ip_addr_changed                0x0000bcbd   Thumb Code    42  udp.o(i.udp_netif_ip_addr_changed)
    udp_new                                  0x0000bced   Thumb Code    28  udp.o(i.udp_new)
    udp_recv                                 0x0000bd61   Thumb Code     6  udp.o(i.udp_recv)
    udp_remove                               0x0000bd69   Thumb Code    64  udp.o(i.udp_remove)
    udp_sendto_if                            0x0000bdad   Thumb Code    82  udp.o(i.udp_sendto_if)
    udp_sendto_if_src                        0x0000be01   Thumb Code   278  udp.o(i.udp_sendto_if_src)
    mcgConfig_BOARD_BootClockRUN             0x0000bf50   Data          11  clock_config.o(.constdata)
    simConfig_BOARD_BootClockRUN             0x0000bf5c   Data           8  clock_config.o(.constdata)
    oscConfig_BOARD_BootClockRUN             0x0000bf64   Data           8  clock_config.o(.constdata)
    mcgConfig_BOARD_BootClockVLPR            0x0000bf6c   Data          11  clock_config.o(.constdata)
    simConfig_BOARD_BootClockVLPR            0x0000bf78   Data           8  clock_config.o(.constdata)
    oscConfig_BOARD_BootClockVLPR            0x0000bf80   Data           8  clock_config.o(.constdata)
    s_enetClock                              0x0000c020   Data           4  fsl_enet.o(.constdata)
    memp_UDP_PCB                             0x0000c02c   Data          16  memp.o(.constdata)
    memp_TCP_PCB                             0x0000c03c   Data          16  memp.o(.constdata)
    memp_TCP_PCB_LISTEN                      0x0000c04c   Data          16  memp.o(.constdata)
    memp_TCP_SEG                             0x0000c05c   Data          16  memp.o(.constdata)
    memp_REASSDATA                           0x0000c06c   Data          16  memp.o(.constdata)
    memp_FRAG_PBUF                           0x0000c07c   Data          16  memp.o(.constdata)
    memp_SYS_TIMEOUT                         0x0000c08c   Data          16  memp.o(.constdata)
    memp_PBUF                                0x0000c09c   Data          16  memp.o(.constdata)
    memp_PBUF_POOL                           0x0000c0ac   Data          16  memp.o(.constdata)
    memp_pools                               0x0000c0bc   Data          36  memp.o(.constdata)
    tcp_pcb_lists                            0x0000c120   Data          16  tcp.o(.constdata)
    lwip_cyclic_timers                       0x0000c130   Data          40  timeouts.o(.constdata)
    ip_addr_any                              0x0000c158   Data           4  ip4_addr.o(.constdata)
    ip_addr_broadcast                        0x0000c15c   Data           4  ip4_addr.o(.constdata)
    ethbroadcast                             0x0000c160   Data           6  ethernet.o(.constdata)
    ethzero                                  0x0000c166   Data           6  ethernet.o(.constdata)
    Region$$Table$$Base                      0x0000c484   Number         0  anon$$obj.o(Region$$Table)
    Region$$Table$$Limit                     0x0000c4a4   Number         0  anon$$obj.o(Region$$Table)
    Image$$VECTOR_RAM$$Base                  0x1fff0000   Number         0  anon$$obj.o ABSOLUTE
    Image$$RW_m_data$$Base                   0x1fff0400   Number         0  anon$$obj.o ABSOLUTE
    SystemCoreClock                          0x20000000   Data           4  system_mk64f12.o(.data)
    g_xtal0Freq                              0x20000010   Data           4  fsl_clock.o(.data)
    g_xtal32Freq                             0x20000014   Data           4  fsl_clock.o(.data)
    errno                                    0x20000030   Data           4  sys_arch.o(.data)
    netif_list                               0x2000006c   Data           4  netif.o(.data)
    netif_default                            0x20000070   Data           4  netif.o(.data)
    tcp_ticks                                0x2000007c   Data           4  tcp.o(.data)
    tcp_bound_pcbs                           0x20000080   Data           4  tcp.o(.data)
    tcp_listen_pcbs                          0x20000084   Data           4  tcp.o(.data)
    tcp_active_pcbs                          0x20000088   Data           4  tcp.o(.data)
    tcp_tw_pcbs                              0x2000008c   Data           4  tcp.o(.data)
    tcp_active_pcbs_changed                  0x20000090   Data           1  tcp.o(.data)
    tcp_input_pcb                            0x200000bc   Data           4  tcp_in.o(.data)
    udp_pcbs                                 0x200000d0   Data           4  udp.o(.data)
    ip_data                                  0x20003730   Data          24  ip.o(.bss)
    ram_heap                                 0x20003748   Data       22547  mem.o(.bss)
    memp_memory_UDP_PCB_base                 0x20008f5b   Data         195  memp.o(.bss)
    memp_memory_TCP_PCB_base                 0x2000901e   Data        1483  memp.o(.bss)
    memp_memory_TCP_PCB_LISTEN_base          0x200095e9   Data         195  memp.o(.bss)
    memp_memory_TCP_SEG_base                 0x200096ac   Data         443  memp.o(.bss)
    memp_memory_REASSDATA_base               0x20009867   Data         163  memp.o(.bss)
    memp_memory_FRAG_PBUF_base               0x2000990a   Data         363  memp.o(.bss)
    memp_memory_SYS_TIMEOUT_base             0x20009a75   Data         163  memp.o(.bss)
    memp_memory_PBUF_base                    0x20009b18   Data         243  memp.o(.bss)
    memp_memory_PBUF_POOL_base               0x20009c0b   Data       13791  memp.o(.bss)
    dhcp_rx_options_val                      0x2000d200   Data          40  dhcp.o(.bss)
    dhcp_rx_options_given                    0x2000d228   Data          10  dhcp.o(.bss)
    Image$$ARM_LIB_STACK$$ZI$$Limit          0x20030000   Number         0  anon$$obj.o ABSOLUTE



==============================================================================

Memory Map of the image

  Image Entry point : 0x00000411

  Load Region LR_m_text (Base: 0x00000000, Size: 0x0000c594, Max: 0x00100000, ABSOLUTE)

    Execution Region VECTOR_ROM (Exec base: 0x00000000, Load base: 0x00000000, Size: 0x00000400, Max: 0x00000400, ABSOLUTE)

    Exec Addr    Load Addr    Size         Type   Attr      Idx    E Section Name        Object

    0x00000000   0x00000000   0x00000400   Data   RO            4    RESET               startup_mk64f12.o


    Execution Region ER_m_flash_config (Exec base: 0x00000400, Load base: 0x00000400, Size: 0x00000010, Max: 0x00000010, ABSOLUTE, FIXED)

    Exec Addr    Load Addr    Size         Type   Attr      Idx    E Section Name        Object

    0x00000400   0x00000400   0x00000010   Data   RO            5    FlashConfig         startup_mk64f12.o


    Execution Region ER_m_text (Exec base: 0x00000410, Load base: 0x00000410, Size: 0x0000c094, Max: 0x000ffbf0, ABSOLUTE)

    Exec Addr    Load Addr    Size         Type   Attr      Idx    E Section Name        Object

    0x00000410   0x00000410   0x00000000   Code   RO         4912  * .ARM.Collect$$$$00000000  mc_w.l(entry.o)
    0x00000410   0x00000410   0x00000004   Code   RO         4929    .ARM.Collect$$$$00000003  mc_w.l(entry4.o)
    0x00000414   0x00000414   0x00000004   Code   RO         4932    .ARM.Collect$$$$00000004  mc_w.l(entry5.o)
    0x00000418   0x00000418   0x00000000   Code   RO         4934    .ARM.Collect$$$$00000008  mc_w.l(entry7b.o)
    0x00000418   0x00000418   0x00000000   Code   RO         4936    .ARM.Collect$$$$0000000A  mc_w.l(entry8b.o)
    0x00000418   0x00000418   0x00000008   Code   RO         4937    .ARM.Collect$$$$0000000B  mc_w.l(entry9a.o)
    0x00000420   0x00000420   0x00000000   Code   RO         4939    .ARM.Collect$$$$0000000D  mc_w.l(entry10a.o)
    0x00000420   0x00000420   0x00000000   Code   RO         4941    .ARM.Collect$$$$0000000F  mc_w.l(entry11a.o)
    0x00000420   0x00000420   0x00000004   Code   RO         4930    .ARM.Collect$$$$00002714  mc_w.l(entry4.o)
    0x00000424   0x00000424   0x000001c4   Code   RO            6    .text               startup_mk64f12.o
    0x000005e8   0x000005e8   0x00000062   Code   RO         4915    .text               mc_w.l(uldiv.o)
    0x0000064a   0x0000064a   0x00000024   Code   RO         4917    .text               mc_w.l(memcpya.o)
    0x0000066e   0x0000066e   0x00000024   Code   RO         4919    .text               mc_w.l(memseta.o)
    0x00000692   0x00000692   0x0000000e   Code   RO         4921    .text               mc_w.l(strlen.o)
    0x000006a0   0x000006a0   0x0000001a   Code   RO         4923    .text               mc_w.l(memcmp.o)
    0x000006ba   0x000006ba   0x0000001e   Code   RO         4943    .text               mc_w.l(llshl.o)
    0x000006d8   0x000006d8   0x00000020   Code   RO         4945    .text               mc_w.l(llushr.o)
    0x000006f8   0x000006f8   0x00000024   Code   RO         4947    .text               mc_w.l(init.o)
    0x0000071c   0x0000071c   0x0000006c   Code   RO          270    i.BOARD_BootClockRUN  clock_config.o
    0x00000788   0x00000788   0x0000001c   Code   RO          229    i.BOARD_InitDebugConsole  board.o
    0x000007a4   0x000007a4   0x000000ec   Code   RO          166    i.BOARD_InitPins    pin_mux.o
    0x00000890   0x00000890   0x0000008c   Code   RO          588    i.CLOCK_BootToPeeMode  fsl_clock.o
    0x0000091c   0x0000091c   0x00000014   Code   RO          272    i.CLOCK_CONFIG_SetFllExtRefDiv  clock_config.o
    0x00000930   0x00000930   0x00000018   Code   RO          167    i.CLOCK_EnableClock  pin_mux.o
    0x00000948   0x00000948   0x00000098   Code   RO          592    i.CLOCK_EnablePll0  fsl_clock.o
    0x000009e0   0x000009e0   0x0000001c   Code   RO          597    i.CLOCK_GetCoreSysClkFreq  fsl_clock.o
    0x000009fc   0x000009fc   0x000000ac   Code   RO          598    i.CLOCK_GetEr32kClkFreq  fsl_clock.o
    0x00000aa8   0x00000aa8   0x0000001c   Code   RO          599    i.CLOCK_GetFixedFreqClkFreq  fsl_clock.o
    0x00000ac4   0x00000ac4   0x00000070   Code   RO          602    i.CLOCK_GetFllExtRefClkFreq  fsl_clock.o
    0x00000b34   0x00000b34   0x0000004c   Code   RO          603    i.CLOCK_GetFllFreq  fsl_clock.o
    0x00000b80   0x00000b80   0x00000020   Code   RO          604    i.CLOCK_GetFllRefClkFreq  fsl_clock.o
    0x00000ba0   0x00000ba0   0x000000c8   Code   RO          605    i.CLOCK_GetFreq     fsl_clock.o
    0x00000c68   0x00000c68   0x0000001c   Code   RO          606    i.CLOCK_GetInternalRefClkFreq  fsl_clock.o
    0x00000c84   0x00000c84   0x0000002c   Code   RO          607    i.CLOCK_GetInternalRefClkSelectFreq  fsl_clock.o
    0x00000cb0   0x00000cb0   0x000000bc   Code   RO          608    i.CLOCK_GetMcgExtClkFreq  fsl_clock.o
    0x00000d6c   0x00000d6c   0x0000007c   Code   RO          610    i.CLOCK_GetOsc0ErClkFreq  fsl_clock.o
    0x00000de8   0x00000de8   0x00000020   Code   RO          611    i.CLOCK_GetOscRangeFromFreq  fsl_clock.o
    0x00000e08   0x00000e08   0x0000003c   Code   RO          612    i.CLOCK_GetOutClkFreq  fsl_clock.o
    0x00000e44   0x00000e44   0x00000090   Code   RO          614    i.CLOCK_GetPll0Freq  fsl_clock.o
    0x00000ed4   0x00000ed4   0x00000008   Code   RO          615    i.CLOCK_GetPll0RefFreq  fsl_clock.o
    0x00000edc   0x00000edc   0x00000038   Code   RO          616    i.CLOCK_GetPllFllSelClkFreq  fsl_clock.o
    0x00000f14   0x00000f14   0x0000006c   Code   RO          618    i.CLOCK_InitOsc0    fsl_clock.o
    0x00000f80   0x00000f80   0x0000003c   Code   RO          622    i.CLOCK_SetExternalRefClkConfig  fsl_clock.o
    0x00000fbc   0x00000fbc   0x00000098   Code   RO          627    i.CLOCK_SetInternalRefClkConfig  fsl_clock.o
    0x00001054   0x00001054   0x000000c4   Code   RO          630    i.CLOCK_SetPbeMode  fsl_clock.o
    0x00001118   0x00001118   0x00000030   Code   RO          634    i.CLOCK_SetSimConfig  fsl_clock.o
    0x00001148   0x00001148   0x000000a8   Code   RO         1707    i.DbgConsole_ConvertRadixNumToString  fsl_debug_console.o
    0x000011f0   0x000011f0   0x00000098   Code   RO         1710    i.DbgConsole_Init   fsl_debug_console.o
    0x00001288   0x00001288   0x00000034   Code   RO         1711    i.DbgConsole_Printf  fsl_debug_console.o
    0x000012bc   0x000012bc   0x0000023a   Code   RO         1712    i.DbgConsole_PrintfFormattedData  fsl_debug_console.o
    0x000014f6   0x000014f6   0x00000028   Code   RO         1713    i.DbgConsole_PrintfPaddingCharacter  fsl_debug_console.o
    0x0000151e   0x0000151e   0x00000002   PAD
    0x00001520   0x00001520   0x00000024   Code   RO         1714    i.DbgConsole_Putchar  fsl_debug_console.o
    0x00001544   0x00001544   0x0000001c   Code   RO          915    i.ENET_1588_Timer_IRQHandler  fsl_enet.o
    0x00001560   0x00001560   0x00000004   Code   RO           80    i.ENET_ClearInterruptStatus  fsl_phy.o
    0x00001564   0x00001564   0x000000b0   Code   RO          919    i.ENET_ErrorIRQHandler  fsl_enet.o
    0x00001614   0x00001614   0x0000001c   Code   RO          920    i.ENET_Error_IRQHandler  fsl_enet.o
    0x00001630   0x00001630   0x0000006c   Code   RO          921    i.ENET_GetDefaultConfig  fsl_enet.o
    0x0000169c   0x0000169c   0x00000090   Code   RO          922    i.ENET_GetInstance  fsl_enet.o
    0x0000172c   0x0000172c   0x000000ec   Code   RO          925    i.ENET_GetRxFrameSize  fsl_enet.o
    0x00001818   0x00001818   0x000002b0   Code   RO          926    i.ENET_Init         fsl_enet.o
    0x00001ac8   0x00001ac8   0x00000124   Code   RO          928    i.ENET_ReadFrame    fsl_enet.o
    0x00001bec   0x00001bec   0x0000007c   Code   RO          929    i.ENET_ReceiveIRQHandler  fsl_enet.o
    0x00001c68   0x00001c68   0x0000001c   Code   RO          930    i.ENET_Receive_IRQHandler  fsl_enet.o
    0x00001c84   0x00001c84   0x000001ac   Code   RO          931    i.ENET_SendFrame    fsl_enet.o
    0x00001e30   0x00001e30   0x000000ac   Code   RO          933    i.ENET_SetHandler   fsl_enet.o
    0x00001edc   0x00001edc   0x0000002c   Code   RO          935    i.ENET_SetMacAddr   fsl_enet.o
    0x00001f08   0x00001f08   0x000001b0   Code   RO          936    i.ENET_SetMacController  fsl_enet.o
    0x000020b8   0x000020b8   0x000000c0   Code   RO          937    i.ENET_SetRxBufferDescriptors  fsl_enet.o
    0x00002178   0x00002178   0x000000a8   Code   RO          938    i.ENET_SetSMI       fsl_enet.o
    0x00002220   0x00002220   0x000000bc   Code   RO          939    i.ENET_SetTxBufferDescriptors  fsl_enet.o
    0x000022dc   0x000022dc   0x0000002c   Code   RO          940    i.ENET_StartSMIRead  fsl_enet.o
    0x00002308   0x00002308   0x00000034   Code   RO          941    i.ENET_StartSMIWrite  fsl_enet.o
    0x0000233c   0x0000233c   0x0000007c   Code   RO          942    i.ENET_TransmitIRQHandler  fsl_enet.o
    0x000023b8   0x000023b8   0x0000001c   Code   RO          943    i.ENET_Transmit_IRQHandler  fsl_enet.o
    0x000023d4   0x000023d4   0x0000008c   Code   RO          944    i.ENET_UpdateReadBuffers  fsl_enet.o
    0x00002460   0x00002460   0x00000024   Code   RO          945    i.EnableIRQ         fsl_enet.o
    0x00002484   0x00002484   0x0000007c   Code   RO           82    i.PHY_GetLinkSpeedDuplex  fsl_phy.o
    0x00002500   0x00002500   0x00000058   Code   RO           83    i.PHY_GetLinkStatus  fsl_phy.o
    0x00002558   0x00002558   0x000000d4   Code   RO           84    i.PHY_Init          fsl_phy.o
    0x0000262c   0x0000262c   0x00000084   Code   RO           85    i.PHY_Read          fsl_phy.o
    0x000026b0   0x000026b0   0x00000058   Code   RO           86    i.PHY_Write         fsl_phy.o
    0x00002708   0x00002708   0x00000068   Code   RO          168    i.PORT_SetPinConfig  pin_mux.o
    0x00002770   0x00002770   0x0000000e   Code   RO          169    i.PORT_SetPinMux    pin_mux.o
    0x0000277e   0x0000277e   0x00000008   Code   RO         1562    i.SysTick_Handler   lwip_dhcp_bm.o
    0x00002786   0x00002786   0x00000002   PAD
    0x00002788   0x00002788   0x0000002c   Code   RO           16    i.SystemInit        system_mk64f12.o
    0x000027b4   0x000027b4   0x0000001c   Code   RO          318    i.UART0_DriverIRQHandler  fsl_uart.o
    0x000027d0   0x000027d0   0x00000008   Code   RO          319    i.UART0_RX_TX_DriverIRQHandler  fsl_uart.o
    0x000027d8   0x000027d8   0x0000001c   Code   RO          320    i.UART1_DriverIRQHandler  fsl_uart.o
    0x000027f4   0x000027f4   0x00000008   Code   RO          321    i.UART1_RX_TX_DriverIRQHandler  fsl_uart.o
    0x000027fc   0x000027fc   0x0000001c   Code   RO          322    i.UART2_DriverIRQHandler  fsl_uart.o
    0x00002818   0x00002818   0x00000008   Code   RO          323    i.UART2_RX_TX_DriverIRQHandler  fsl_uart.o
    0x00002820   0x00002820   0x0000001c   Code   RO          324    i.UART3_DriverIRQHandler  fsl_uart.o
    0x0000283c   0x0000283c   0x00000008   Code   RO          325    i.UART3_RX_TX_DriverIRQHandler  fsl_uart.o
    0x00002844   0x00002844   0x0000001c   Code   RO          326    i.UART4_DriverIRQHandler  fsl_uart.o
    0x00002860   0x00002860   0x00000008   Code   RO          327    i.UART4_RX_TX_DriverIRQHandler  fsl_uart.o
    0x00002868   0x00002868   0x0000001c   Code   RO          328    i.UART5_DriverIRQHandler  fsl_uart.o
    0x00002884   0x00002884   0x00000008   Code   RO          329    i.UART5_RX_TX_DriverIRQHandler  fsl_uart.o
    0x0000288c   0x0000288c   0x00000070   Code   RO          334    i.UART_GetDefaultConfig  fsl_uart.o
    0x000028fc   0x000028fc   0x0000008c   Code   RO          336    i.UART_GetInstance  fsl_uart.o
    0x00002988   0x00002988   0x00000018   Code   RO          337    i.UART_GetStatusFlags  fsl_uart.o
    0x000029a0   0x000029a0   0x000002a4   Code   RO          338    i.UART_Init         fsl_uart.o
    0x00002c44   0x00002c44   0x000000b0   Code   RO          339    i.UART_ReadBlocking  fsl_uart.o
    0x00002cf4   0x00002cf4   0x00000020   Code   RO          355    i.UART_WriteBlocking  fsl_uart.o
    0x00002d14   0x00002d14   0x00000044   Code   RO         1125    i.__aeabi_assert    fsl_common.o
    0x00002d58   0x00002d58   0x0000000e   Code   RO         4951    i.__scatterload_copy  mc_w.l(handlers.o)
    0x00002d66   0x00002d66   0x00000002   Code   RO         4952    i.__scatterload_null  mc_w.l(handlers.o)
    0x00002d68   0x00002d68   0x0000000e   Code   RO         4953    i.__scatterload_zeroinit  mc_w.l(handlers.o)
    0x00002d76   0x00002d76   0x00000002   PAD
    0x00002d78   0x00002d78   0x0000001c   Code   RO         3425    i.cyclic_timer      timeouts.o
    0x00002d94   0x00002d94   0x0000004c   Code   RO         3644    i.dhcp_arp_reply    dhcp.o
    0x00002de0   0x00002de0   0x00000164   Code   RO         3645    i.dhcp_bind         dhcp.o
    0x00002f44   0x00002f44   0x0000004c   Code   RO         3646    i.dhcp_check        dhcp.o
    0x00002f90   0x00002f90   0x00000078   Code   RO         3648    i.dhcp_coarse_tmr   dhcp.o
    0x00003008   0x00003008   0x0000025c   Code   RO         3649    i.dhcp_create_msg   dhcp.o
    0x00003264   0x00003264   0x00000060   Code   RO         3650    i.dhcp_dec_pcb_refcount  dhcp.o
    0x000032c4   0x000032c4   0x000000a8   Code   RO         3651    i.dhcp_decline      dhcp.o
    0x0000336c   0x0000336c   0x000000b4   Code   RO         3652    i.dhcp_delete_msg   dhcp.o
    0x00003420   0x00003420   0x000000f4   Code   RO         3653    i.dhcp_discover     dhcp.o
    0x00003514   0x00003514   0x00000040   Code   RO         3654    i.dhcp_fine_tmr     dhcp.o
    0x00003554   0x00003554   0x00000080   Code   RO         3655    i.dhcp_handle_ack   dhcp.o
    0x000035d4   0x000035d4   0x0000002c   Code   RO         3656    i.dhcp_handle_nak   dhcp.o
    0x00003600   0x00003600   0x00000040   Code   RO         3657    i.dhcp_handle_offer  dhcp.o
    0x00003640   0x00003640   0x000000a8   Code   RO         3658    i.dhcp_inc_pcb_refcount  dhcp.o
    0x000036e8   0x000036e8   0x0000003c   Code   RO         3661    i.dhcp_option       dhcp.o
    0x00003724   0x00003724   0x00000060   Code   RO         3662    i.dhcp_option_byte  dhcp.o
    0x00003784   0x00003784   0x00000094   Code   RO         3663    i.dhcp_option_long  dhcp.o
    0x00003818   0x00003818   0x00000038   Code   RO         3664    i.dhcp_option_short  dhcp.o
    0x00003850   0x00003850   0x000000f8   Code   RO         3665    i.dhcp_option_trailer  dhcp.o
    0x00003948   0x00003948   0x00000428   Code   RO         3666    i.dhcp_parse_reply  dhcp.o
    0x00003d70   0x00003d70   0x000000d0   Code   RO         3667    i.dhcp_rebind       dhcp.o
    0x00003e40   0x00003e40   0x000000ec   Code   RO         3668    i.dhcp_reboot       dhcp.o
    0x00003f2c   0x00003f2c   0x00000184   Code   RO         3669    i.dhcp_recv         dhcp.o
    0x000040b0   0x000040b0   0x000000b8   Code   RO         3670    i.dhcp_release      dhcp.o
    0x00004168   0x00004168   0x000000d0   Code   RO         3671    i.dhcp_renew        dhcp.o
    0x00004238   0x00004238   0x00000114   Code   RO         3672    i.dhcp_select       dhcp.o
    0x0000434c   0x0000434c   0x00000010   Code   RO         3673    i.dhcp_set_state    dhcp.o
    0x0000435c   0x0000435c   0x00000128   Code   RO         3675    i.dhcp_start        dhcp.o
    0x00004484   0x00004484   0x00000070   Code   RO         3676    i.dhcp_stop         dhcp.o
    0x000044f4   0x000044f4   0x00000022   Code   RO         3677    i.dhcp_supplied_address  dhcp.o
    0x00004516   0x00004516   0x0000004a   Code   RO         3678    i.dhcp_t1_timeout   dhcp.o
    0x00004560   0x00004560   0x00000050   Code   RO         3679    i.dhcp_t2_timeout   dhcp.o
    0x000045b0   0x000045b0   0x00000088   Code   RO         3680    i.dhcp_timeout      dhcp.o
    0x00004638   0x00004638   0x00000054   Code   RO         2516    i.do_memp_free_pool  memp.o
    0x0000468c   0x0000468c   0x00000064   Code   RO         2517    i.do_memp_malloc_pool  memp.o
    0x000046f0   0x000046f0   0x00000010   Code   RO         1822    i.enet_get_rx_frame_size  ethernetif.o
    0x00004700   0x00004700   0x0000000c   Code   RO         1823    i.enet_get_tx_buffer  ethernetif.o
    0x0000470c   0x0000470c   0x000000c8   Code   RO         1824    i.enet_init         ethernetif.o
    0x000047d4   0x000047d4   0x00000016   Code   RO         1825    i.enet_read_frame   ethernetif.o
    0x000047ea   0x000047ea   0x00000034   Code   RO         1826    i.enet_send_frame   ethernetif.o
    0x0000481e   0x0000481e   0x00000002   PAD
    0x00004820   0x00004820   0x00000260   Code   RO         3872    i.etharp_find_entry  etharp.o
    0x00004a80   0x00004a80   0x00000078   Code   RO         3873    i.etharp_free_entry  etharp.o
    0x00004af8   0x00004af8   0x00000124   Code   RO         3875    i.etharp_input      etharp.o
    0x00004c1c   0x00004c1c   0x0000017c   Code   RO         3876    i.etharp_output     etharp.o
    0x00004d98   0x00004d98   0x000000fc   Code   RO         3877    i.etharp_output_to_arp_index  etharp.o
    0x00004e94   0x00004e94   0x00000218   Code   RO         3878    i.etharp_query      etharp.o
    0x000050ac   0x000050ac   0x0000010c   Code   RO         3879    i.etharp_raw        etharp.o
    0x000051b8   0x000051b8   0x0000001c   Code   RO         3880    i.etharp_request    etharp.o
    0x000051d4   0x000051d4   0x0000002c   Code   RO         3881    i.etharp_request_dst  etharp.o
    0x00005200   0x00005200   0x000000e4   Code   RO         3882    i.etharp_tmr        etharp.o
    0x000052e4   0x000052e4   0x000000fc   Code   RO         3883    i.etharp_update_arp_entry  etharp.o
    0x000053e0   0x000053e0   0x000000dc   Code   RO         4384    i.ethernet_input    ethernet.o
    0x000054bc   0x000054bc   0x000000a0   Code   RO         4385    i.ethernet_output   ethernet.o
    0x0000555c   0x0000555c   0x0000005c   Code   RO         1827    i.ethernetif_init   ethernetif.o
    0x000055b8   0x000055b8   0x00000044   Code   RO         1828    i.ethernetif_input  ethernetif.o
    0x000055fc   0x000055fc   0x00000012   Code   RO         3970    i.icmp_dest_unreach  icmp.o
    0x0000560e   0x0000560e   0x00000002   PAD
    0x00005610   0x00005610   0x00000274   Code   RO         3971    i.icmp_input        icmp.o
    0x00005884   0x00005884   0x000000bc   Code   RO         3972    i.icmp_send_response  icmp.o
    0x00005940   0x00005940   0x00000012   Code   RO         3973    i.icmp_time_exceeded  icmp.o
    0x00005952   0x00005952   0x00000014   Code   RO         2276    i.inet_chksum       inet_chksum.o
    0x00005966   0x00005966   0x00000052   Code   RO         2277    i.inet_chksum_pbuf  inet_chksum.o
    0x000059b8   0x000059b8   0x0000004c   Code   RO         2278    i.inet_chksum_pseudo  inet_chksum.o
    0x00005a04   0x00005a04   0x00000086   Code   RO         2280    i.inet_cksum_pseudo_base  inet_chksum.o
    0x00005a8a   0x00005a8a   0x0000004e   Code   RO         4079    i.ip4_addr_isbroadcast_u32  ip4_addr.o
    0x00005ad8   0x00005ad8   0x00000240   Code   RO         4144    i.ip4_frag          ip4_frag.o
    0x00005d18   0x00005d18   0x00000248   Code   RO         4029    i.ip4_input         ip4.o
    0x00005f60   0x00005f60   0x00000036   Code   RO         4031    i.ip4_output_if     ip4.o
    0x00005f96   0x00005f96   0x00000002   PAD
    0x00005f98   0x00005f98   0x00000168   Code   RO         4032    i.ip4_output_if_src  ip4.o
    0x00006100   0x00006100   0x000001c4   Code   RO         4145    i.ip4_reass         ip4_frag.o
    0x000062c4   0x000062c4   0x00000094   Code   RO         4033    i.ip4_route         ip4.o
    0x00006358   0x00006358   0x00000024   Code   RO         2282    i.ip_chksum_pseudo  inet_chksum.o
    0x0000637c   0x0000637c   0x0000000a   Code   RO         4146    i.ip_frag_alloc_pbuf_custom_ref  ip4_frag.o
    0x00006386   0x00006386   0x00000002   PAD
    0x00006388   0x00006388   0x00000028   Code   RO         4147    i.ip_frag_free_pbuf_custom_ref  ip4_frag.o
    0x000063b0   0x000063b0   0x00000270   Code   RO         4148    i.ip_reass_chain_frag_into_datagram_and_validate  ip4_frag.o
    0x00006620   0x00006620   0x00000050   Code   RO         4149    i.ip_reass_dequeue_datagram  ip4_frag.o
    0x00006670   0x00006670   0x00000058   Code   RO         4150    i.ip_reass_enqueue_new_datagram  ip4_frag.o
    0x000066c8   0x000066c8   0x00000140   Code   RO         4151    i.ip_reass_free_complete_datagram  ip4_frag.o
    0x00006808   0x00006808   0x00000088   Code   RO         4152    i.ip_reass_remove_oldest_datagram  ip4_frag.o
    0x00006890   0x00006890   0x0000003c   Code   RO         4153    i.ip_reass_tmr      ip4_frag.o
    0x000068cc   0x000068cc   0x0000004c   Code   RO         4154    i.ipfrag_free_pbuf_custom  ip4_frag.o
    0x00006918   0x00006918   0x0000004c   Code   RO         1829    i.low_level_init    ethernetif.o
    0x00006964   0x00006964   0x000000ae   Code   RO         1830    i.low_level_input   ethernetif.o
    0x00006a12   0x00006a12   0x00000002   PAD
    0x00006a14   0x00006a14   0x000000a0   Code   RO         1831    i.low_level_output  ethernetif.o
    0x00006ab4   0x00006ab4   0x0000001a   Code   RO         2203    i.lwip_htonl        def.o
    0x00006ace   0x00006ace   0x0000000c   Code   RO         2204    i.lwip_htons        def.o
    0x00006ada   0x00006ada   0x00000020   Code   RO         2359    i.lwip_init         init.o
    0x00006afa   0x00006afa   0x0000005e   Code   RO         2284    i.lwip_standard_chksum  inet_chksum.o
    0x00006b58   0x00006b58   0x00000100   Code   RO         1563    i.main              lwip_dhcp_bm.o
    0x00006c58   0x00006c58   0x000000e0   Code   RO         2457    i.mem_free          mem.o
    0x00006d38   0x00006d38   0x0000005c   Code   RO         2458    i.mem_init          mem.o
    0x00006d94   0x00006d94   0x000001ec   Code   RO         2459    i.mem_malloc        mem.o
    0x00006f80   0x00006f80   0x00000170   Code   RO         2460    i.mem_trim          mem.o
    0x000070f0   0x000070f0   0x0000004c   Code   RO         2518    i.memp_free         memp.o
    0x0000713c   0x0000713c   0x00000020   Code   RO         2520    i.memp_init         memp.o
    0x0000715c   0x0000715c   0x0000002c   Code   RO         2521    i.memp_init_pool    memp.o
    0x00007188   0x00007188   0x0000004c   Code   RO         2522    i.memp_malloc       memp.o
    0x000071d4   0x000071d4   0x000000b4   Code   RO         2610    i.netif_add         netif.o
    0x00007288   0x00007288   0x00000002   Code   RO         2612    i.netif_init        netif.o
    0x0000728a   0x0000728a   0x00000024   Code   RO         2614    i.netif_issue_reports  netif.o
    0x000072ae   0x000072ae   0x00000048   Code   RO         2616    i.netif_set_addr    netif.o
    0x000072f6   0x000072f6   0x00000002   PAD
    0x000072f8   0x000072f8   0x00000010   Code   RO         2617    i.netif_set_default  netif.o
    0x00007308   0x00007308   0x00000010   Code   RO         2619    i.netif_set_gw      netif.o
    0x00007318   0x00007318   0x00000054   Code   RO         2620    i.netif_set_ipaddr  netif.o
    0x0000736c   0x0000736c   0x00000010   Code   RO         2623    i.netif_set_netmask  netif.o
    0x0000737c   0x0000737c   0x0000002c   Code   RO         2624    i.netif_set_up      netif.o
    0x000073a8   0x000073a8   0x00000364   Code   RO         2733    i.pbuf_alloc        pbuf.o
    0x0000770c   0x0000770c   0x000000b0   Code   RO         2734    i.pbuf_alloced_custom  pbuf.o
    0x000077bc   0x000077bc   0x000000d0   Code   RO         2735    i.pbuf_cat          pbuf.o
    0x0000788c   0x0000788c   0x0000001a   Code   RO         2736    i.pbuf_chain        pbuf.o
    0x000078a6   0x000078a6   0x00000012   Code   RO         2737    i.pbuf_clen         pbuf.o
    0x000078b8   0x000078b8   0x00000198   Code   RO         2739    i.pbuf_copy         pbuf.o
    0x00007a50   0x00007a50   0x000000e4   Code   RO         2740    i.pbuf_copy_partial  pbuf.o
    0x00007b34   0x00007b34   0x00000140   Code   RO         2742    i.pbuf_free         pbuf.o
    0x00007c74   0x00007c74   0x00000012   Code   RO         2744    i.pbuf_header       pbuf.o
    0x00007c86   0x00007c86   0x00000012   Code   RO         2745    i.pbuf_header_force  pbuf.o
    0x00007c98   0x00007c98   0x000000f4   Code   RO         2746    i.pbuf_header_impl  pbuf.o
    0x00007d8c   0x00007d8c   0x00000140   Code   RO         2750    i.pbuf_realloc      pbuf.o
    0x00007ecc   0x00007ecc   0x0000001e   Code   RO         2751    i.pbuf_ref          pbuf.o
    0x00007eea   0x00007eea   0x00000002   PAD
    0x00007eec   0x00007eec   0x0000013c   Code   RO         2461    i.plug_holes        mem.o
    0x00008028   0x00008028   0x00000200   Code   RO         1564    i.print_dhcp_state  lwip_dhcp_bm.o
    0x00008228   0x00008228   0x00000012   Code   RO         1971    i.sys_arch_protect  sys_arch.o
    0x0000823a   0x0000823a   0x0000000e   Code   RO         1972    i.sys_arch_unprotect  sys_arch.o
    0x00008248   0x00008248   0x00000018   Code   RO         1973    i.sys_assert        sys_arch.o
    0x00008260   0x00008260   0x0000006c   Code   RO         3426    i.sys_check_timeouts  timeouts.o
    0x000082cc   0x000082cc   0x0000000c   Code   RO         1974    i.sys_now           sys_arch.o
    0x000082d8   0x000082d8   0x00000120   Code   RO         3428    i.sys_timeout       timeouts.o
    0x000083f8   0x000083f8   0x00000034   Code   RO         3429    i.sys_timeouts_init  timeouts.o
    0x0000842c   0x0000842c   0x00000134   Code   RO         2953    i.tcp_abandon       tcp.o
    0x00008560   0x00008560   0x0000000e   Code   RO         2954    i.tcp_abort         tcp.o
    0x0000856e   0x0000856e   0x00000002   PAD
    0x00008570   0x00008570   0x000000d4   Code   RO         2957    i.tcp_alloc         tcp.o
    0x00008644   0x00008644   0x00000064   Code   RO         2959    i.tcp_backlog_accepted  tcp.o
    0x000086a8   0x000086a8   0x00000020   Code   RO         2962    i.tcp_close         tcp.o
    0x000086c8   0x000086c8   0x000001e0   Code   RO         2963    i.tcp_close_shutdown  tcp.o
    0x000088a8   0x000088a8   0x000000f0   Code   RO         3315    i.tcp_create_segment  tcp_out.o
    0x00008998   0x00008998   0x0000003a   Code   RO         2966    i.tcp_eff_send_mss_impl  tcp.o
    0x000089d2   0x000089d2   0x00000002   PAD
    0x000089d4   0x000089d4   0x0000020c   Code   RO         3316    i.tcp_enqueue_flags  tcp_out.o
    0x00008be0   0x00008be0   0x0000007c   Code   RO         2968    i.tcp_fasttmr       tcp.o
    0x00008c5c   0x00008c5c   0x00000058   Code   RO         3244    i.tcp_getoptbyte    tcp_in.o
    0x00008cb4   0x00008cb4   0x00000002   Code   RO         2969    i.tcp_init          tcp.o
    0x00008cb6   0x00008cb6   0x00000002   PAD
    0x00008cb8   0x00008cb8   0x00000718   Code   RO         3245    i.tcp_input         tcp_in.o
    0x000093d0   0x000093d0   0x0000008a   Code   RO         3317    i.tcp_keepalive     tcp_out.o
    0x0000945a   0x0000945a   0x00000002   PAD
    0x0000945c   0x0000945c   0x0000005c   Code   RO         2970    i.tcp_kill_prio     tcp.o
    0x000094b8   0x000094b8   0x00000070   Code   RO         2971    i.tcp_kill_state    tcp.o
    0x00009528   0x00009528   0x00000040   Code   RO         2972    i.tcp_kill_timewait  tcp.o
    0x00009568   0x00009568   0x00000064   Code   RO         2973    i.tcp_listen_closed  tcp.o
    0x000095cc   0x000095cc   0x00000168   Code   RO         3246    i.tcp_listen_input  tcp_in.o
    0x00009734   0x00009734   0x00000054   Code   RO         2975    i.tcp_netif_ip_addr_changed  tcp.o
    0x00009788   0x00009788   0x0000002e   Code   RO         2976    i.tcp_netif_ip_addr_changed_pcblist  tcp.o
    0x000097b6   0x000097b6   0x00000002   PAD
    0x000097b8   0x000097b8   0x0000001c   Code   RO         2980    i.tcp_next_iss      tcp.o
    0x000097d4   0x000097d4   0x00000278   Code   RO         3318    i.tcp_output        tcp_out.o
    0x00009a4c   0x00009a4c   0x000000bc   Code   RO         3319    i.tcp_output_alloc_header  tcp_out.o
    0x00009b08   0x00009b08   0x000000e4   Code   RO         3320    i.tcp_output_segment  tcp_out.o
    0x00009bec   0x00009bec   0x000000b8   Code   RO         3247    i.tcp_parseopt      tcp_in.o
    0x00009ca4   0x00009ca4   0x0000005e   Code   RO         2981    i.tcp_pcb_purge     tcp.o
    0x00009d02   0x00009d02   0x00000002   PAD
    0x00009d04   0x00009d04   0x000000c0   Code   RO         2982    i.tcp_pcb_remove    tcp.o
    0x00009dc4   0x00009dc4   0x00000690   Code   RO         3248    i.tcp_process       tcp_in.o
    0x0000a454   0x0000a454   0x0000009a   Code   RO         2984    i.tcp_process_refused_data  tcp.o
    0x0000a4ee   0x0000a4ee   0x00000002   PAD
    0x0000a4f0   0x0000a4f0   0x000007ec   Code   RO         3249    i.tcp_receive       tcp_in.o
    0x0000acdc   0x0000acdc   0x0000002e   Code   RO         2986    i.tcp_recv_null     tcp.o
    0x0000ad0a   0x0000ad0a   0x00000002   PAD
    0x0000ad0c   0x0000ad0c   0x000000c4   Code   RO         2987    i.tcp_recved        tcp.o
    0x0000add0   0x0000add0   0x00000018   Code   RO         2988    i.tcp_remove_listener  tcp.o
    0x0000ade8   0x0000ade8   0x0000005a   Code   RO         3322    i.tcp_rexmit        tcp_out.o
    0x0000ae42   0x0000ae42   0x0000007c   Code   RO         3323    i.tcp_rexmit_fast   tcp_out.o
    0x0000aebe   0x0000aebe   0x00000044   Code   RO         3324    i.tcp_rexmit_rto    tcp_out.o
    0x0000af02   0x0000af02   0x00000002   PAD
    0x0000af04   0x0000af04   0x000000dc   Code   RO         3325    i.tcp_rst           tcp_out.o
    0x0000afe0   0x0000afe0   0x0000001a   Code   RO         2989    i.tcp_seg_free      tcp.o
    0x0000affa   0x0000affa   0x00000018   Code   RO         2990    i.tcp_segs_free     tcp.o
    0x0000b012   0x0000b012   0x00000096   Code   RO         3326    i.tcp_send_empty_ack  tcp_out.o
    0x0000b0a8   0x0000b0a8   0x0000004a   Code   RO         3327    i.tcp_send_fin      tcp_out.o
    0x0000b0f2   0x0000b0f2   0x00000002   PAD
    0x0000b0f4   0x0000b0f4   0x00000544   Code   RO         2994    i.tcp_slowtmr       tcp.o
    0x0000b638   0x0000b638   0x00000038   Code   RO         3432    i.tcp_timer_needed  timeouts.o
    0x0000b670   0x0000b670   0x000000a4   Code   RO         3250    i.tcp_timewait_input  tcp_in.o
    0x0000b714   0x0000b714   0x00000024   Code   RO         2995    i.tcp_tmr           tcp.o
    0x0000b738   0x0000b738   0x00000014   Code   RO         3251    i.tcp_trigger_input_pcb_close  tcp_in.o
    0x0000b74c   0x0000b74c   0x00000078   Code   RO         2997    i.tcp_update_rcv_ann_wnd  tcp.o
    0x0000b7c4   0x0000b7c4   0x00000106   Code   RO         3330    i.tcp_zero_window_probe  tcp_out.o
    0x0000b8ca   0x0000b8ca   0x00000002   PAD
    0x0000b8cc   0x0000b8cc   0x00000038   Code   RO         3433    i.tcpip_tcp_timer   timeouts.o
    0x0000b904   0x0000b904   0x00000074   Code   RO         1975    i.time_init         sys_arch.o
    0x0000b978   0x0000b978   0x00000010   Code   RO         1976    i.time_isr          sys_arch.o
    0x0000b988   0x0000b988   0x000000b4   Code   RO         3505    i.udp_bind          udp.o
    0x0000ba3c   0x0000ba3c   0x0000007c   Code   RO         3506    i.udp_connect       udp.o
    0x0000bab8   0x0000bab8   0x00000002   Code   RO         3508    i.udp_init          udp.o
    0x0000baba   0x0000baba   0x00000002   PAD
    0x0000babc   0x0000babc   0x000001b8   Code   RO         3509    i.udp_input         udp.o
    0x0000bc74   0x0000bc74   0x00000048   Code   RO         3510    i.udp_input_local_match  udp.o
    0x0000bcbc   0x0000bcbc   0x00000030   Code   RO         3511    i.udp_netif_ip_addr_changed  udp.o
    0x0000bcec   0x0000bcec   0x0000001c   Code   RO         3512    i.udp_new           udp.o
    0x0000bd08   0x0000bd08   0x00000058   Code   RO         3514    i.udp_new_port      udp.o
    0x0000bd60   0x0000bd60   0x00000006   Code   RO         3515    i.udp_recv          udp.o
    0x0000bd66   0x0000bd66   0x00000002   PAD
    0x0000bd68   0x0000bd68   0x00000044   Code   RO         3516    i.udp_remove        udp.o
    0x0000bdac   0x0000bdac   0x00000052   Code   RO         3519    i.udp_sendto_if     udp.o
    0x0000bdfe   0x0000bdfe   0x00000002   PAD
    0x0000be00   0x0000be00   0x00000148   Code   RO         3520    i.udp_sendto_if_src  udp.o
    0x0000bf48   0x0000bf48   0x00000006   Data   RO          170    .constdata          pin_mux.o
    0x0000bf4e   0x0000bf4e   0x00000002   PAD
    0x0000bf50   0x0000bf50   0x00000038   Data   RO          273    .constdata          clock_config.o
    0x0000bf88   0x0000bf88   0x00000038   Data   RO          358    .constdata          fsl_uart.o
    0x0000bfc0   0x0000bfc0   0x00000060   Data   RO          636    .constdata          fsl_clock.o
    0x0000c020   0x0000c020   0x0000000c   Data   RO          946    .constdata          fsl_enet.o
    0x0000c02c   0x0000c02c   0x000000b4   Data   RO         2525    .constdata          memp.o
    0x0000c0e0   0x0000c0e0   0x00000050   Data   RO         2998    .constdata          tcp.o
    0x0000c130   0x0000c130   0x00000028   Data   RO         3434    .constdata          timeouts.o
    0x0000c158   0x0000c158   0x00000008   Data   RO         4086    .constdata          ip4_addr.o
    0x0000c160   0x0000c160   0x0000000c   Data   RO         4386    .constdata          ethernet.o
    0x0000c16c   0x0000c16c   0x00000115   Data   RO          947    .conststring        fsl_enet.o
    0x0000c281   0x0000c281   0x00000003   PAD
    0x0000c284   0x0000c284   0x00000068   Data   RO         2526    .conststring        memp.o
    0x0000c2ec   0x0000c2ec   0x0000006d   Data   RO         2999    .conststring        tcp.o
    0x0000c359   0x0000c359   0x00000003   PAD
    0x0000c35c   0x0000c35c   0x00000055   Data   RO         3331    .conststring        tcp_out.o
    0x0000c3b1   0x0000c3b1   0x00000003   PAD
    0x0000c3b4   0x0000c3b4   0x0000008c   Data   RO         3682    .conststring        dhcp.o
    0x0000c440   0x0000c440   0x00000041   Data   RO         3885    .conststring        etharp.o
    0x0000c481   0x0000c481   0x00000003   PAD
    0x0000c484   0x0000c484   0x00000020   Data   RO         4949    Region$$Table       anon$$obj.o


    Execution Region VECTOR_RAM (Exec base: 0x1fff0000, Load base: 0x0000c4a4, Size: 0x00000400, Max: 0x00000400, ABSOLUTE)

    Exec Addr    Load Addr    Size         Type   Attr      Idx    E Section Name        Object

    0x1fff0000        -       0x00000400   Zero   RW            1    VECTOR_RAM.bss      anon$$obj.o


    Execution Region RW_m_data (Exec base: 0x1fff0400, Load base: 0x0000c4a4, Size: 0x00000000, Max: 0x0000fc00, ABSOLUTE)

    **** No section assigned to this execution region ****


    Execution Region RW_m_data_2 (Exec base: 0x20000000, Load base: 0x0000c4a4, Size: 0x0000d324, Max: 0x0002e000, ABSOLUTE)

    Exec Addr    Load Addr    Size         Type   Attr      Idx    E Section Name        Object

    0x20000000   0x0000c4a4   0x00000004   Data   RW           17    .data               system_mk64f12.o
    0x20000004   0x0000c4a8   0x00000004   Data   RW          359    .data               fsl_uart.o
    0x20000008   0x0000c4ac   0x00000010   Data   RW          637    .data               fsl_clock.o
    0x20000018   0x0000c4bc   0x00000014   Data   RW          948    .data               fsl_enet.o
    0x2000002c   0x0000c4d0   0x00000001   Data   RW         1565    .data               lwip_dhcp_bm.o
    0x2000002d   0x0000c4d1   0x00000003   PAD
    0x20000030   0x0000c4d4   0x0000000c   Data   RW         1977    .data               sys_arch.o
    0x2000003c   0x0000c4e0   0x0000000c   Data   RW         2463    .data               mem.o
    0x20000048   0x0000c4ec   0x00000024   Data   RW         2527    .data               memp.o
    0x2000006c   0x0000c510   0x00000009   Data   RW         2625    .data               netif.o
    0x20000075   0x0000c519   0x00000003   PAD
    0x20000078   0x0000c51c   0x00000020   Data   RW         3000    .data               tcp.o
    0x20000098   0x0000c53c   0x00000028   Data   RW         3253    .data               tcp_in.o
    0x200000c0   0x0000c564   0x0000000c   Data   RW         3435    .data               timeouts.o
    0x200000cc   0x0000c570   0x00000008   Data   RW         3521    .data               udp.o
    0x200000d4   0x0000c578   0x00000010   Data   RW         3683    .data               dhcp.o
    0x200000e4   0x0000c588   0x00000001   Data   RW         3886    .data               etharp.o
    0x200000e5   0x0000c589   0x00000001   PAD
    0x200000e6   0x0000c58a   0x00000002   Data   RW         4034    .data               ip4.o
    0x200000e8   0x0000c58c   0x00000006   Data   RW         4155    .data               ip4_frag.o
    0x200000ee   0x0000c592   0x00000002   PAD
    0x200000f0        -       0x00000018   Zero   RW          357    .bss                fsl_uart.o
    0x20000108        -       0x00000010   Zero   RW         1720    .bss                fsl_debug_console.o
    0x20000118        -       0x00003616   Zero   RW         1832    .bss                ethernetif.o
    0x2000372e   0x0000c592   0x00000002   PAD
    0x20003730        -       0x00000018   Zero   RW         2432    .bss                ip.o
    0x20003748        -       0x00005813   Zero   RW         2462    .bss                mem.o
    0x20008f5b        -       0x0000428f   Zero   RW         2524    .bss                memp.o
    0x2000d1ea   0x0000c592   0x00000002   PAD
    0x2000d1ec        -       0x00000014   Zero   RW         3252    .bss                tcp_in.o
    0x2000d200        -       0x00000032   Zero   RW         3681    .bss                dhcp.o
    0x2000d232   0x0000c592   0x00000002   PAD
    0x2000d234        -       0x000000f0   Zero   RW         3884    .bss                etharp.o


    Execution Region ARM_LIB_HEAP (Exec base: 0x2000d324, Load base: 0x0000c594, Size: 0x00001000, Max: 0x00001000, ABSOLUTE)

    Exec Addr    Load Addr    Size         Type   Attr      Idx    E Section Name        Object

    0x2000d324        -       0x00001000   Zero   RW            2    ARM_LIB_HEAP.bss    anon$$obj.o


    Execution Region ARM_LIB_STACK (Exec base: 0x2002f000, Load base: 0x0000c594, Size: 0x00001000, Max: 0x00001000, ABSOLUTE)

    Exec Addr    Load Addr    Size         Type   Attr      Idx    E Section Name        Object

    0x2002f000        -       0x00001000   Zero   RW            3    ARM_LIB_STACK.bss   anon$$obj.o


==============================================================================

Image component sizes


      Code (inc. data)   RO Data    RW Data    ZI Data      Debug   Object Name

        28          4          0          0          0        553   board.o
       128         36         56          0          0      10027   clock_config.o
        38          0          0          0          0       1274   def.o
      6308       1240        140         16         50      32980   dhcp.o
      3008        512         65          1        240      12352   etharp.o
       380         56         12          0          0       3022   ethernet.o
       872         82          0          0      13846      35216   ethernetif.o
      2188        696         96         16          0      28942   fsl_clock.o
        68         44          0          0          0       8309   fsl_common.o
      1018         26          0          0         16      14705   fsl_debug_console.o
      3900       1390        289         20          0      31006   fsl_enet.o
       648         94          0          0          0      24344   fsl_phy.o
      1376        538         56          4         24      52680   fsl_uart.o
       852        158          0          0          0       4526   icmp.o
       442          0          0          0          0      13080   inet_chksum.o
        32          0          0          0          0      14154   init.o
         0          0          0          0         24       3134   ip.o
      1146         90          0          2          0       5824   ip4.o
        78          0          8          0          0       7338   ip4_addr.o
      2462        492          0          6          0      11970   ip4_frag.o
       776        434          0          1          0      19548   lwip_dhcp_bm.o
      1492        488          0         12      22547       6025   mem.o
       412        148        284         36      17039      11658   memp.o
       466         42          0          9          0      10138   netif.o
      2882       1004          0          0          0      12831   pbuf.o
       378         96          6          0          0     477096   pin_mux.o
       452        212       1040          0          0       3360   startup_mk64f12.o
       200         30          0         12          0      31209   sys_arch.o
        44         10          0          4          0     469811   system_mk64f12.o
      4116        858        189         32          0      32311   tcp.o
      6340       1038          0         40         20      19791   tcp_in.o
      2938        372         85          0          0      13811   tcp_out.o
       588        138         40         12          0       6531   timeouts.o
      1466        118          0          8          0      12929   udp.o

    ----------------------------------------------------------------------
     47568      10446       2412        240      63028    1442485   Object Totals
         0          0         32          0       9216          0   (incl. Generated)
        46          0         14          9          6          0   (incl. Padding)

    ----------------------------------------------------------------------

      Code (inc. data)   RO Data    RW Data    ZI Data      Debug   Library Member Name

         0          0          0          0          0          0   entry.o
         0          0          0          0          0          0   entry10a.o
         0          0          0          0          0          0   entry11a.o
         8          4          0          0          0          0   entry4.o
         4          0          0          0          0          0   entry5.o
         0          0          0          0          0          0   entry7b.o
         0          0          0          0          0          0   entry8b.o
         8          4          0          0          0          0   entry9a.o
        30          0          0          0          0          0   handlers.o
        36          8          0          0          0         68   init.o
        30          0          0          0          0         68   llshl.o
        32          0          0          0          0         68   llushr.o
        26          0          0          0          0         80   memcmp.o
        36          0          0          0          0         68   memcpya.o
        36          0          0          0          0        108   memseta.o
        14          0          0          0          0         68   strlen.o
        98          0          0          0          0         92   uldiv.o

    ----------------------------------------------------------------------
       360         16          0          0          0        620   Library Totals
         2          0          0          0          0          0   (incl. Padding)

    ----------------------------------------------------------------------

      Code (inc. data)   RO Data    RW Data    ZI Data      Debug   Library Name

       358         16          0          0          0        620   mc_w.l

    ----------------------------------------------------------------------
       360         16          0          0          0        620   Library Totals

    ----------------------------------------------------------------------

==============================================================================


      Code (inc. data)   RO Data    RW Data    ZI Data      Debug   

     47928      10462       2412        240      63028    1415901   Grand Totals
     47928      10462       2412        240      63028    1415901   ELF Image Totals
     47928      10462       2412        240          0          0   ROM Totals

==============================================================================

    Total RO  Size (Code + RO Data)                50340 (  49.16kB)
    Total RW  Size (RW Data + ZI Data)             63268 (  61.79kB)
    Total ROM Size (Code + RO Data + RW Data)      50580 (  49.39kB)

==============================================================================

